:1000000000400020D550000015510000175100009D
:1000100000000000000000000000000000000000E0
:100020000000000000000000000000001951000066
:1000300000000000000000001B5100001D510000E6
:100040001F510000D9380000515500001F51000019
:100050001F510000000000001F5100001F51000050
:100060001F510000155800001F5100001F510000D3
:100070001F5100001F5100001F5100001F510000C0
:100080001F510000AD5900001F5100001F5100001A
:100090001F5100001F5100001F5100001F510000A0
:1000A0001F5100001F510000000000000000000070
:1000B0000000000000000000000000000000000040
:1000C00010B5064C2378002B07D1054B002B02D02E
:1000D000044800E000BF0123237010BD4802002047
:1000E0000000000040B70000044B10B5002B03D007
:1000F0000349044800E000BF10BDC04600000000F6
:100100004C02002040B70000164B002B00D1144BCE
:100110009D46402292029A1A924600218B460F4633
:100120001348144A121A08F082FD0F4B002B00D01E
:1001300098470E4B002B00D0984700200021040068
:100140000D000D48002802D00C4800E000BF08F068
:100150002DFD2000290005F013FA08F001FDC0462E
:100160000000080000400020000000000000000027
:1001700048020020C8250020000000000000000008
:1001800002000120104004D1042A01D9106800099E
:1001900070470020FCE710B50400FFF7F1FF0028CE
:1001A00009D001388000031D22181279002A02D0DC
:1001B00001309842F8D110BD0122096810B51142F2
:1001C00001D0002903DA102000F084F910BD491095
:1001D000062002F011F8F9E7096810B5CB0701D540
:1001E000002903DA102000F075F910BD4910033121
:1001F00089100022052001F0FFFFF6E770B50D68B9
:10020000AB0729D1042D27D90F232A684E68134044
:10021000062B0BD12800FFF7B3FF0123984201DA28
:1002200000200AE09A00AE500133F7E7052B13D106
:10023000F30703D4132000F04DF970BD7610FF2EA4
:10024000F8D82800FFF79CFF2C1D80002018A04242
:10025000E6D926700134FAE70B2000F03BF9DFE71E
:1002600070B50C681120E30712D54D68AB072BD190
:10027000042D29D90F262B6864101E40062E0DD19F
:10028000002C04DD2800FFF77BFFA04203DA1220D8
:1002900000F020F901E0A400605970BD331F012B6C
:1002A00012D82800FFF76CFF8000042E02D128002E
:1002B000FFF771FF002CEADDA042E8DB01202C19DA
:1002C000E3785B001843E8E70B20E1E7F8B501238A
:1002D0000D6811201D4214D003244E6834402CD1E7
:1002E000042E2AD90F2332686D108F681340062B15
:1002F0000ED1002D04DD3000FFF742FFA84203DAE3
:10030000122000F0E7F802E0AD00AF512000F8BD88
:10031000052B12D1002DF3DD3000FFF731FF8000F7
:10032000A842EDDB01231F4201D11320E9E77F1032
:10033000FF2FFAD87519EF70E8E70B20E1E708689E
:1003400010B5830717D1042815D90F23026813406D
:10035000062B03D1FFF714FF430004E0052B05D162
:10036000FFF70EFFC3000120184310BD042B02D17C
:10037000FFF711FFF0E70B2000F0ACF8F5E7000005
:1003800002000120104001D0501070470D22014B97
:100390001A70FAE78802002002000120104004D100
:1003A000042A01D91068000970470020FCE770B5E5
:1003B0000E000400FFF7F0FF05003000FFF7ECFF30
:1003C0000023854206D10434AD0004366519AC42E1
:1003D00002D30123180070BD20783278002801D1A3
:1003E000002AF6D0013401369042F0D00023F1E724
:1003F000F0B585B00393019002912D4E2D4B002A4C
:1004000002D002223270013A00251A601B68F554AE
:10041000019B9D4201DB05B0F0BD029AAB00D058B4
:10042000244B1C68C8239B0037191C1B012318424E
:1004300006D0214A43102100380008F0A1FF09E04E
:100440001E4A002802D004281BD11D4A2100380072
:1004500008F096FF300008F0F7FF164A039B106083
:10046000002B0CD0019B013BAB4208DD154B9842A1
:1004700005D8431C1360202232540022F254013567
:10048000C6E7042810D90F2302681340042B04D1B7
:1004900001F0EEFE0C4A0300CDE7062B05D1FFF775
:1004A0007BFF0A4A0300C6E70123094AC3E7C046A7
:1004B00089020020AC050020D5A30000A8A30000FD
:1004C000AEA300001F030000C7AF0000B3A30000ED
:1004D000C4A30000014B1870002070478802002060
:1004E00070B501F0E7FC094C0100251D1F22280012
:1004F00008F0B1FF280008F0A7FF042304308008AB
:10050000000118432060200070BDC0466402002036
:10051000C368F0B59D00836889B05D190300183386
:1005200006930369069A9F00069B0390DF194369AF
:1005300001939B00D3180293CD4B1B78002B26D13F
:100540007F222B68CB491C1213409B005B5804355B
:1005500001929F46039B587803F05AFE0023039AAA
:10056000137027E0C24B1B78002B10D12B68019A27
:100570001C121340BF4A9B009B580435E9E7069BB9
:100580003A1DD11ABA4BD82928DD1A221A70039BBA
:10059000B74C9B6821780193EA1A039B92109B78D1
:1005A00012021A43039B587803F03AFE0023039A81
:1005B00023701370039B069A9B680193ED1A039BAB
:1005C000AD10DD60069BFE1A039BB6101E61029BF8
:1005D0009B1A039A9B10536109B0F0BD1B783C60D5
:1005E000002B01D01700D2E72B6801991C120B4099
:1005F000A0499B005B5817000435AAE7069B3A1DEB
:10060000D11A9B4BD82902DD1A221A70BFE728683D
:100610001B78291D3860002B02D017000D00B6E7AB
:100620006B6801991C120B4092499B005B581700A4
:1006300008358EE7069B3A1DD11A8D4BD82902DD6D
:100640001A221A70A3E7A4001B782C193C60002B17
:1006500001D017009BE72B6801991C120B408549BC
:100660009B005B581700043573E7069B3A1DD11AAF
:100670007F4BD82902DD1A221A7088E77E49A40030
:1006800061581B783960002B01D017007FE72B6879
:1006900001991C120B4077499B005B5817000435E9
:1006A00057E7043F744B3A68A400E250704B1B7844
:1006B000002B00D06BE72B68019A1C1213406D4A87
:1006C0009B009B58043544E76B4BA400E058FFF7B0
:1006D00057FE043F06003868FFF752FE3618012027
:1006E000654B76000643E650614B1B78002B00D02B
:1006F0004DE72B68019A1C1213405E4A9B009B58E1
:10070000043526E7069B3A1DD11A594BD82902DD3C
:100710001A221A703BE70698029C0121A04202D2DD
:1007200021000C3909681B783960002B01D01700B3
:100730002DE72B6801991C120B404E499B005B581A
:100740001700043505E7069B3A1DD11A484BD829F6
:1007500002DD1A221A701AE70699029881420FD216
:1007600003000C3B1B6845495B106418E41AA400A5
:1007700023583B603E4B1B78002B05D0170006E743
:10078000182119700023F4E72B6801991C120B4003
:1007900038499B005B5817000435DAE6069B029A3D
:1007A000934219D213000C3B1B68344A043FA4182F
:1007B0005B10E31A029A39689B0099502C4B1B7806
:1007C000002B00D0E3E62B68019A1C121340294A43
:1007D0009B009B580435BCE61822254B1A70EDE7A8
:1007E000069B029A93422DD2244B3E1FE31814001D
:1007F0000C3C04932368049A5B10D31A029A9B0062
:100800009858FFF7BDFD07903068FFF7B9FD2468E1
:10081000049B64101C1B079BA4001F1801207F0071
:10082000029B0743E7503700114B1B78002B00D089
:10083000ADE62B68019A1C1213400E4A9B009B5890
:10084000043586E618220A4B1A70EDE7069B3A1D1E
:10085000D11A074BD82902DD1A221A7097E602999D
:10086000A40061581B783960002B09D017008EE670
:1008700088020020A8A1000070230020FDFFFF3F98
:100880002B6801991C120B40D8499B005B5817003C
:1008900004355EE6043F029B3A68A400E250D44B64
:1008A0001B78002B00D072E62B68019A1C121340B3
:1008B000CE4A9B009B5804354BE6029BA4001C19B2
:1008C0002368043F38685E10FFF75AFD3618012090
:1008D000C74B76001B7806432660002B00D056E6F7
:1008E0002B68019A1C121340C04A9B009B58043588
:1008F0002FE6069BA4003F1BBD4CBB420CD82378BF
:10090000002B00D043E62B68019A1C121340B74A13
:100910009B009B5804351CE6B64801F01DFC23786B
:10092000002B00D033E62B68019A1C121340AF4A0B
:100930009B009B5804350CE6A300ED18002C00DA50
:1009400038E6AB4B1B78002B00D020E62B68019AD1
:100950001C121340A54A9B009B580435F9E5043F3F
:100960003B68042B04D1A300ED18002C00DA21E62B
:100970009F4B1B78002B00D009E62B68019A1C12B4
:1009800013409A4A9B009B580435E2E5043F3B68BC
:10099000042B06D0A200AD18002C02DA002B00D1E7
:1009A00008E6934B1B78002B00D0F0E52B68019AEA
:1009B0001C1213408D4A9B009B580435C9E53A1F11
:1009C00013685B10013B002B06DD01215B00A400D6
:1009D0000B432D191360EDE5854B17001B78002B99
:1009E00000D0D4E52B68019A1C1213407F4A9B006B
:1009F0009B580435ADE53A00069B0C32D31AD82B30
:100A000003DD1A227A4B1A70C1E5FF2361005B00F7
:100A10001940FE3BFF3B19433960039906988968EA
:100A2000241204916D1A0399AD1089782D020D439B
:100A300002999D40091A891099401D430B43BB60E0
:100A4000039B7D609C70E4B26B4BE4000292E35820
:100A5000039A9360664A1278002A03D008331D0077
:100A6000029F94E51D00019A9B680C351C121340EF
:100A70005E4A9B009B58029F6BE53B1F1C68029AD5
:100A8000069B93422FD10A20E3070ED4A30715D16A
:100A9000042C13D90F2322681340042B11D12000FA
:100AA00001F0E6FB08F0D0FC0630643003F09AF861
:100AB00000280FD1043D069B02937BE50720042C00
:100AC000F3D02000431E9841FA234042FF331840E0
:100AD0000730EAE7039B2100587803F0B3FB0023BB
:100AE000039A1370E7E7029B029A0C3B1B68039979
:100AF0005B109B00D31A0C3B1C601F1D1300083BAE
:100B00001B685A108A70D2B23B49D2005B0055581C
:100B10009B0A039A9B009560ED18029B069A043B82
:100B20001B685B109B00D3180293314B1B78002B82
:100B300000D02CE52B68019A1C1213402B4A9B0015
:100B40009B58043505E53B1F1868FFF719FCA40006
:100B500006003F1B1E2827DC00280DDC244B1B78D9
:100B6000002B00D013E52B68019A1C1213401F4A7A
:100B70009B009B580435ECE401F08AF9033E3618DB
:100B800001F086F91D4B801B9842F9D8184B1B7851
:100B9000002B00D0FBE42B68019A1C121340134A6F
:100BA0009B009B580435D4E40123039A137001F091
:100BB0006FF9039B0A3886195E60FBE43B1F1868D7
:100BC000FFF7DEFBA40006003F1B002818DC084BE3
:100BD0001B78002B00D0DAE42B68019A1C1213401A
:100BE000024A9B009B580435B3E4C046A8A100000C
:100BF00088020020D8A30000781B00209F860100F7
:100C0000C64B984203DD1D22C54B1A70BFE4012379
:100C1000039A137001F03CF9FA239B005E43039B97
:100C20000A3E30185860C5E4A300FF1A00232000D4
:100C30001A003900FFF7DCFBBA4EBB4C31682000CC
:100C400003F0B8F93168200003F003FB316820009D
:100C500001F0A4FBB24B1B78002B00D097E42B686B
:100C6000019A1C121340B14A9B009B58043570E452
:100C7000AB4BA4001B783F1B002B00D087E42B68F4
:100C8000019A1C121340A94A9B009B58043560E44A
:100C9000039803F00BF8A24B1B78002B00D076E4EE
:100CA0002B68019A1C121340A04A9B009B580435E4
:100CB0004FE43B1F1868002838D1083B1868C30769
:100CC0001ED540103A0001234100083A0B4313603F
:100CD000002859DD01234200391F1A430A603A00F7
:100CE000083A12681A41101A3A000C3A116819426F
:100CF0001FD0C0189840A4001843029BE05027E082
:100D000083070FD104280DD90F2302681340062B47
:100D100002D1FFF741FBD5E7052B03D1FFF73CFBE1
:100D20008000CFE719227E4B1A7030E44010013862
:100D3000CEE78A0723D1042921D90F220E68324039
:100D4000062A15D1013080004358029AA400A3500E
:100D5000734B1B78002B01D0FFF719FC2B68019A0D
:100D60001C121340714A9B009B580435FFF7F1FB9E
:100D7000052A04D108180079A4004000BCE7192214
:100D8000674B1A70FFF703FC0435E1E7A300069AEE
:100D9000FB189B1AD82B13DC0122631E002C14DCD9
:100DA0005F4B1B78002B01D0FFF7F1FB2B68019AFA
:100DB0001C1213405D4A9B009B580435FFF7C9FB8A
:100DC0001A22574B1A70FFF7E2FB3A601C000437F7
:100DD000E3E7069A3B1D9B1A514ED82B03DD1A23DD
:100DE0003370FFF7D4FB069B029AA40093422AD2E9
:100DF0003B1F1868FFF7C4FA011E21DD029B0C3B64
:100E00001A68521082421BDB9007801A484B401828
:100E1000C018029B8000C2583B1B1A60404B3F1B0E
:100E20001B780437002B01D0FFF7B1FB2B68019A28
:100E30001C1213403D4A9B009B580435FFF789FB69
:100E400020233370EAE71823FBE7A3009C46FE1A31
:100E5000002C17DC1C22324B1A70002333606346CF
:100E6000FF1A2F4B04371B78002B01D0FFF78FFBA5
:100E70002B68019A1C1213402C4A9B009B58043586
:100E8000FFF767FB002033685A108300F1580123F5
:100E90000B4003D10D21224A1170DFE749108A422D
:100EA00000DD0A0001308442EFDC012352001343CD
:100EB000D4E7A3009C46FE1A002C17DC1C22184B1A
:100EC0001A70002333606346FF1A154B04371B78F2
:100ED000002B01D0FFF75BFB2B68019A1C1213401B
:100EE000124A9B009B580435FFF733FB0020336800
:100EF0005A108300F15801230B4003D10D21084AF9
:100F00001170DFE749108A4200DA0A00013084429A
:100F1000EFDC012352001343D4E7C04680EE3600D5
:100F200088020020AC05002089020020A8A1000052
:100F3000FCFFFF3F3B00083B1868FFF721FA3B1F0F
:100F400006001868FFF71CFA0023864200DA043313
:100F5000A4003A1B17001360E34B04371B78002BE7
:100F600001D0FFF714FB2B68019A1C121340DF4AD3
:100F70009B009B580435FFF7ECFA3B00083B1868D0
:100F8000FFF7FEF93B1F06001868FFF7F9F9F30FAA
:100F9000C217B0425341A4003A1B17009B001360D4
:100FA000D14B04371B78002B01D0FFF7F0FA2B68E8
:100FB000019A1C121340CD4A9B009B580435FFF741
:100FC000C8FA3B00083B18683B1F1968A600BE1B07
:100FD0000423814202D0042802D8002333601CE09D
:100FE0000123184201D01942F7D103239C4618422D
:100FF000F3D102680C331A40042AEED16246114242
:10100000EBD10429E9D90A681340042BE5D1FFF795
:10101000CEF9431E984180003060B34BA4001B788A
:101020003F1B0437002B01D0FFF7B1FA2B68019A60
:101030001C121340AD4A9B009B580435FFF789FAF8
:101040003B00083B18683B1F1968A600BE1B002325
:10105000814202D0042802D8042333601CE001231B
:10106000184201D01942F7D103239C461842F3D10C
:1010700002680C331A40042AEED162461142EBD1C9
:101080000429E9D90A681340042BE5D1FFF78FF949
:101090004342584180003060934BA4001B783F1BB3
:1010A0000437002B01D0FFF772FA2B68019A1C124B
:1010B00013408E4A9B009B580435FFF74AFA3B00C9
:1010C000083B1868FFF75CF93B1F06001868FFF73C
:1010D00057F9F317C20F86425341A4003A1B170079
:1010E0009B001360804B04371B78002B01D0FFF767
:1010F0004EFA2B68019A1C1213407C4A9B009B58A5
:101100000435FFF726FA3B00083B1868FFF738F96B
:101110003B1F06001868FFF733F90023864200DD05
:101120000433A4003A1B170013606F4B04371B787D
:10113000002B01D0FFF72BFA2B68019A1C121340E9
:101140006A4A9B009B580435FFF703FA3B1F1B6854
:10115000A400043B5A1E93413A1B17009B001360E6
:10116000614B04371B78002B01D0FFF710FA2B6876
:10117000019A1C1213405D4A9B009B580435FFF7EF
:10118000E8F93B00083B1868FFF7FAF83B1F060038
:101190001868FFF7F5F832180120A4003B1B1F0068
:1011A000520002431A60504B04371B78002B01D0C9
:1011B000FFF7EDF92B68019A1C1213404B4A9B0074
:1011C0009B580435FFF7C5F93B00083B1868FFF74B
:1011D000D7F83B1F06001868FFF7D2F8321A012033
:1011E000A4003B1B1F00520002431A603E4B043711
:1011F0001B78002B01D0FFF7CAF92B68019A1C124B
:1012000013403A4A9B009B580435FFF7A2F93B0074
:10121000083B1868FFF7B4F83B1F06001868FFF793
:10122000AFF802000120A4003B1B1F0072435200D4
:1012300002431A602C4B04371B78002B01D0FFF7B8
:10124000A6F92B68019A1C121340284A9B009B5850
:101250000435FFF77EF93B1F1868FFF791F8061E6B
:1012600017D11F22204B1A70A4003B1B1F001E60C9
:101270001D4B04371B78002B01D0FFF788F92B6832
:10128000019A1C121340194A9B009B580435FFF722
:1012900060F93B00083B1868FFF772F8310005F071
:1012A000A5FE012640000643DEE73B1F1868FFF756
:1012B00067F8061E1CD11F220B4B1A70A4003B1BA3
:1012C0001F001E60084B04371B78002B01D0FFF76E
:1012D0005EF92B68019A1C121340044A9B009B582C
:1012E0000435FFF736F9C04688020020A8A10000A7
:1012F0003B00083B1868FFF743F8310005F05CFF3E
:10130000012649000E43D9E73B1F1868FFF738F85C
:10131000C217801850400122A4003B1B1F00400050
:1013200010431860F14B04371B78002B01D0FFF7F6
:101330002EF92B68019A1C121340ED4A9B009B5812
:101340000435FFF706F9A300FE1A3068012C24D1FA
:10135000FFF716F80494079007F0CEFF07990029CD
:1013600000DC012105F028FF049BA400C91801231B
:1013700049001943DD4B3F1B1B7831600437002BBC
:1013800001D0FFF704F92B68019A1C121340D84AC8
:101390009B009B580435FFF7DCF8FEF7F1FF049043
:1013A0007068FEF7EDFF049B0130C31A0793D3E783
:1013B000A300FE1A31002000049300F08FFF049B6D
:1013C0003060FF1AC94B04371B78002B01D0FFF7A0
:1013D000DEF82B68019A1C121340C54A9B009B58EB
:1013E0000435FFF7B6F83B00083B1868FEF7C8FF66
:1013F0003B1F06001868FEF7C3FF02000120A4008F
:101400003B1B1F003240520002431A60B74B0437A7
:101410001B78002B01D0FFF7BAF82B68019A1C1239
:101420001340B34A9B009B580435FFF792F83B00EA
:10143000083B1868FEF7A4FF06003B1F1868FEF77C
:101440009FFF320002430120A4003B1B1F005200FB
:1014500002431A60A54B04371B78002B01D0FFF71D
:1014600096F82B68019A1C121340A14A9B009B58C6
:101470000435FFF76EF83B00083B1868FEF780FF65
:1014800006003B1F1868FEF77BFF32004240012038
:10149000A4003B1B1F00520002431A60934B043709
:1014A0001B78002B01D0FFF772F82B68019A1C12F1
:1014B00013408F4A9B009B580435FFF74AF83B1FA7
:1014C0001868FEF75DFFC0430122A4003B1B1F000C
:1014D000400010431860854B04371B78002B01D067
:1014E000FFF755F82B68019A1C121340804A9B00A5
:1014F0009B580435FFF72DF83B00083B1868FEF7B2
:101500003FFF06003B1F1868FEF73AFF320082409B
:1015100051000122A4003B1B1F000A431A60734BB9
:1015200004371B78002B01D0FFF731F82B68019AA4
:101530001C1213406E4A9B009B580435FFF709F8B4
:101540003B00083B1868FEF71BFF06003B1F1868AE
:10155000FEF716FF3200024151000122A4003B1B9E
:101560001F000A431A60614B04371B78002B01D01F
:10157000FFF70DF82B68019A1C1213405C4A9B0080
:101580009B580435FEF7E5FF3B000C3B1868FEF75F
:10159000F7FE3B00083B06001868FEF7F1FEF11766
:1015A0000200C317300005F059FE3B1F049005915F
:1015B0001868FEF7E5FE02000498059905F002FEA2
:1015C00043000120A4003E1B37001843474B306006
:1015D0001B780437002B01D0FEF7D9FF2B68019A46
:1015E0001C121340424A9B009B580435FEF7B1FF82
:1015F000A300FE1A310020000493FEF7DDFD049BDA
:101600003060FF1A394B04371B78002B01D0FEF7EE
:10161000BEFF2B68019A1C121340354A9B009B5851
:101620000435FEF796FFA300FE1A31002000049354
:10163000FEF7D2FD049B3060FF1A2C4B04371B7859
:10164000002B01D0FEF7A3FF2B68019A1C12134058
:10165000274A9B009B580435FEF77BFFA300FF1A27
:1016600039002000FEF7CAFD204B1B78002B01D06B
:10167000FEF78DFF2B68019A1C1213401C4A9B0039
:101680009B580435FEF765FFA300FE1A31002000C9
:101690000493FEF7E5FD049B3060FF1A134B0437FB
:1016A0001B78002B01D0FEF772FF2B68019A1C12E9
:1016B00013400F4A9B009B580435FEF74AFFA300D6
:1016C000FF1A39002000FEF701FE084B1B78002BA3
:1016D00001D0FEF75CFF2B68019A1C121340044AEC
:1016E0009B009B580435FEF734FFC046880200205B
:1016F000A8A10000A300FE1A310020000493FEF709
:101700001EFE049B3060FF1AF14B04371B78002B40
:1017100001D0FEF73CFF2B68019A1C121340ED4AE2
:101720009B009B580435FEF714FF069B3E1DF31AE1
:10173000E74CD82B03DD1A232370FEF728FF00F0B7
:10174000B1FB43000120184323783860002B02D0FE
:101750003700FEF71CFF2B68019A1C121340DD4A6C
:101760009B009B5837000435FEF7F3FE069B3E1D99
:10177000F31AD74CD82B03DD1A232370FEF707FF8B
:1017800000F086FBD44B4000184001231843237817
:101790003860002B02D03700FEF7F9FE2B68019A63
:1017A0001C121340CB4A9B009B5837000435FEF7B0
:1017B000D0FE0123A600BE1B20001A003100FEF758
:1017C00017FEC64C2068643002F00CFA002802D1E3
:1017D000043DFEF7EFFE039B21685A78C04802F0F3
:1017E00046FD0123039A3700137000F051FBBD4BF7
:1017F00022681B68063253431818039B5860FEF793
:10180000D9FEA600BE1B2000012300223100FEF7F6
:10181000EFFDB24C2068643002F0E4F90028D7D024
:10182000AF4802F01FFBDCE7A4003E1BFEF758FEAA
:101830003700A74B30601B780437002B01D0FEF730
:10184000A6FE2B68019A1C121340A24A9B009B58CB
:101850000435FEF77EFEA4003E1B300000F050FB76
:1018600037009B4B30601B780437002B01D0FEF70C
:101870008EFE2B68019A1C121340964A9B009B58BF
:101880000435FEF766FEA4003E1B300000F03AFB74
:1018900037008F4B30601B780437002B01D0FEF7E8
:1018A00076FE2B68019A1C1213408A4A9B009B58B3
:1018B0000435FEF74EFEA4003E1B300000F024FB72
:1018C0003700834B30601B780437002B01D0FEF7C4
:1018D0005EFE2B68019A1C1213407E4A9B009B58A7
:1018E0000435FEF736FEA4003F1B380000F02AFB4B
:1018F000774B1B78002B01D0FEF749FE2B68019A2D
:101900001C121340734A9B009B580435FEF721FEBE
:10191000A300FE1A31002000049300F033FB049B67
:101920003060FF1A6A4B04371B78002B01D0FEF79A
:101930002EFE2B68019A1C121340664A9B009B588E
:101940000435FEF706FEA4003F1B380000F054FBF0
:101950005F4B1B78002B01D0FEF719FE2B68019A14
:101960001C1213405B4A9B009B580435FEF7F1FDA7
:101970000121200000F028FB554B1B78002B01D0E3
:10198000FEF705FE2B68019A1C121340514A9B007A
:101990009B580435FEF7DDFD0021200000F014FB0C
:1019A0004B4B1B78002B01D0FEF7F1FD2B68019A01
:1019B0001C121340474A9B009B580435FEF7C9FD93
:1019C000A4003E1B300000F033FB3700404B30607A
:1019D0001B780437002B01D0FEF7D9FD2B68019A44
:1019E0001C1213403B4A9B009B580435FEF7B1FD87
:1019F000A4003E1B300000F02FFB3700344B30605A
:101A00001B780437002B01D0FEF7C1FD2B68019A2B
:101A10001C1213402F4A9B009B580435FEF799FD7A
:101A2000A4003F1B380000F0F1FA294B1B78002B73
:101A300001D0FEF7ACFD2B68019A1C121340254A19
:101A40009B009B580435FEF784FDA4003F1B380023
:101A500002F0F4FE1E4B1B78002B01D0FEF797FD21
:101A60002B68019A1C1213401A4A9B009B5804359C
:101A7000FEF76FFDA4003E1B300002F071FF37003F
:101A8000134B30601B780437002B01D0FEF77FFD2D
:101A90002B68019A1C1213400E4A9B009B58043578
:101AA000FEF757FDA4003F1B380002F077FE084BFD
:101AB0001B78002B01D0FEF76AFD2B68019A1C12DF
:101AC0001340044A9B009B580435FEF742FDC04674
:101AD00088020020A8A10000FEFFFF7FAC050020C7
:101AE0008902002004000020A4003E1B300002F008
:101AF0006BFE3700B14B30601B780437002B01D0F0
:101B0000FEF745FD2B68019A1C121340AC4A9B005E
:101B10009B580435FEF71DFDA300FF1A3900200075
:101B200000F0B0FEA54B1B78002B01D0FEF72FFD77
:101B30002B68019A1C121340A14A9B009B58043544
:101B4000FEF707FDA300FF1A3900200000F024FD76
:101B50009A4B1B78002B01D0FEF719FD2B68019AD8
:101B60001C121340964A9B009B580435FEF7F1FC6B
:101B7000A300FF1A3900200000F01EFD8F4B1B78D8
:101B8000002B01D0FEF703FD2B68019A1C121340B5
:101B90008B4A9B009B580435FEF7DBFCA300FF1A21
:101BA0003900200000F030FD844B1B78002B01D061
:101BB000FEF7EDFC2B68019A1C121340804A9B0033
:101BC0009B580435FEF7C5FCA300FE1A3100200027
:101BD000049302F04FFF049B3060FF1A774B0437E9
:101BE0001B78002B01D0FEF7D2FC2B68019A1C1247
:101BF0001340734A9B009B580435FEF7AAFCA300D0
:101C0000FE1A31002000049302F03CFF049B306078
:101C1000FF1A6A4B04371B78002B01D0FEF7B7FC84
:101C20002B68019A1C121340654A9B009B5804358F
:101C3000FEF78FFCA300FE1A31002000049302F08F
:101C400029FF049B3060FF1A5C4B04371B78002B84
:101C500001D0FEF79CFC2B68019A1C121340584AD5
:101C60009B009B580435FEF774FCA300FE1A31005C
:101C70002000049302F04AFD049B3060FF1A4F4B92
:101C800004371B78002B01D0FEF781FC2B68019AEA
:101C90001C1213404A4A9B009B580435FEF759FC1E
:101CA000A300FF1A3900200000F08EFD434B1B7883
:101CB000002B01D0FEF76BFC2B68019A1C1213401D
:101CC0003F4A9B009B580435FEF743FCA300FF1AD4
:101CD0003900200000F0C0FC384B1B78002B01D0ED
:101CE000FEF755FC2B68019A1C121340344A9B00E6
:101CF0009B580435FEF72DFCA300FE1A310020008E
:101D0000049300F0D5FD049B3060FF1A2B4B043781
:101D10001B78002B01D0FEF73AFC2B68019A1C12AD
:101D20001340274A9B009B580435FEF712FCA30082
:101D3000FF1A3900200000F02FFD204B1B78002BEC
:101D400001D0FEF724FC2B68019A1C1213401C4A98
:101D50009B009B580435FEF7FCFBA300FF1A3900DB
:101D6000200001F0C5FE154B1B78002B01D0FEF7BB
:101D70000EFC2B68019A1C121340114A9B009B58C1
:101D80000435FEF7E6FBA300FE1A310020000493A1
:101D900001F0AEFE049B3060FF1A084B04371B783D
:101DA000002B01D0FEF7F3FB2B68019A1C121340A5
:101DB000034A9B009B580435FEF7CBFB88020020AA
:101DC000A8A100000023F7B55A1E0192002B07DAE4
:101DD00000F0A2FD02F048F902F0A0FA642301939A
:101DE00000263000194B1968B14212DD184B1A68F1
:101DF00001328A420FDAF0241A601D68154F6C43D5
:101E0000E35D002B1FD0E419022B06D12000FEF762
:101E10007FFB019BD8E70022EDE7012B0DD10028C5
:101E200001D100F035F8F0226A43BB185B680A491B
:101E3000C31A8B4201D80223BB54F0235D43054BE8
:101E4000EB5C022BE2D00136CCE7C046B0050020A7
:101E500000000020181200209F860100002070471B
:101E600000207047002070470020704701220020AA
:101E7000054B06491A615850043103305850083157
:101E8000801858501A607047008000400405000018
:101E90000122034B1A64A822D20098587047C0460A
:101EA0000080004010B5FFF7F3FFFA21890005F02C
:101EB00013F810BD0048704728A400001D2070478B
:101EC00070B5054E0400335C0D008B4202D003F068
:101ED000EDFC355570BDC046B405002070B500243A
:101EE000064D635D012B05D10021200003F0DEFCCF
:101EF0000023635501341D2CF2D170BDB4050020C0
:101F00000D2070473B207047036870B55B100120BF
:101F1000052B12D8094A9B009C58094D2B5D002BBC
:101F200005D00021200003F0C1FC00232B55200028
:101F300003F06AFB43000120184370BD10A40000A9
:101F4000B4050020036870B55D101C2D14D80B4E2D
:101F50004468735D012B05D00121280003F0A6FC25
:101F600001237355064964108C4202DCE143C91712
:101F70002140280003F0CEFB70BDC046B405002010
:101F8000FF0300000B6870B55D101C2D16D80024EF
:101F9000012804DD4C68043C63425C416400094E46
:101FA000735DA34204D02100280003F07FFC745528
:101FB000280003F0AFFC0423012800D00023180000
:101FC00070BDC046B405002070B504000D001C288B
:101FD0000ED8084E335C012B04D0012103F066FCBF
:101FE00001233355290020004D1EA94103F07CFC3C
:101FF00070BDC046B405002010B543680068191FC5
:102000004B4259414010FFF7DFFF10BD37B569461D
:102010000A00064B30CB30C203680220042B02D1E9
:1020200000F0CAFA37BD00F0EFFAFBE7E8A30000C2
:1020300010B5084C6379002B05D00021052003F072
:1020400035FC00236371052003F064FC43425841D2
:10205000800010BDB405002010B5084CE37A002BB9
:1020600005D000210B2003F021FC0023E3720B209C
:1020700003F050FC43425841800010BDB4050020DD
:102080007047704710B5034A0421034801F01CFD56
:1020900010BDC046F0A3000000AB0000E12110B568
:1020A0004902094803F0AEF8FFF7E0FE0A2003F00A
:1020B000A5FA0023FF21054A995401331D2BFBD1BA
:1020C00000F076FD10BDC046A0110020B405002030
:1020D000F8B50B4E070030000D0003F0DBF80400EC
:1020E000A84200DD2C003D00EB1B9C4205DD3000CA
:1020F00003F0DAF828700135F6E72000F8BDC04695
:10210000A011002010B50100014803F083F810BDB4
:10211000A011002010B5054C200003F089F8E12142
:102120002000490203F06EF810BDC046A011002047
:10213000064B01201A68064B06491A6000239A00D4
:1021400001338850642BFAD17047C046DC0500206B
:10215000D40500207023002000B59BB00200054983
:1021600001A807F03FF901A801F098FE02F0D6F8A7
:10217000FCE7C046AFA4000037B5184D040028683E
:10218000002801D006F040FDA400200006F032FD3A
:102190002860002802D11248FFF7DEFF01AB984209
:1021A00007D2104B02196B440193934201D20E489F
:1021B000F2E7042802D808302860083C2B680B4A54
:1021C0001C1913600A4B01201C60002309499A0066
:1021D00001338850642BFAD137BDC046DC0500209E
:1021E00055A400001CFCFFFF85A40000D4050020BE
:1021F000D80500207023002070B50D4D0D4E040051
:102200004B1C28689B003668C318B34203D90A20C8
:10221000FEF760F970BD2B600500AB4205D80F23B7
:1022200009011C4021430160F4E704C5F5E7C046FD
:10223000D4050020D80500200322CB1C70B50C006B
:10224000D9171140C9180500891000220420FFF792
:10225000D3FF0023A34206DBE343DB171C4000232C
:102260000419237170BDE95CC21811710133F1E7E3
:1022700010B5830706D1042804D90F2208C81340DB
:10228000042B03D00E20FEF725F9014810BDC046EF
:10229000BFA4000010B501240B681C4016D05C10D0
:1022A000200005F037F90B4905F002F806F0CAFBEB
:1022B00003F074FC0022084B05F09AFD03F016FCB5
:1022C00006F050FB43000120184310BD0D20FEF71F
:1022D00001F9E5E7D30237390000D04010B50324F7
:1022E0000868044006D1042804D90F23026813406B
:1022F000042B03D00E20FEF7EDF810BDFFF7B8FF5A
:1023000003782100233B5A4253411022C01807F0A2
:1023100039F980239B05C218044B9A4201D9142035
:10232000E9E7430001201843E7E7C046FFFFFF3F0E
:1023300010B5034A0221034801F0C6FB10BDC04698
:10234000C8A40000C0A400000020704710B51E20E3
:10235000FEF7C0F810BD10B51E20FEF7BBF810BD8B
:1023600010B51E20FEF7B6F810BD10B51E20FEF702
:10237000B1F810BD10B51E20FEF7ACF810BD10B5B9
:102380001E20FEF7A7F810BD10B51E20FEF7A2F81C
:1023900010BD10B51E20FEF79DF810BD704700005F
:1023A00010B5034A0921034801F08EFB10BDC04659
:1023B000E8A4000030A500000120034B1860034B87
:1023C0001B68834018437047F4050020E005002097
:1023D000F0B5EFF310810123194083F31088134CFB
:1023E000134AA4461268134E013A9340124F134AFF
:1023F000002B17D0146803420FD03D682C60C046F4
:10240000C046C046C046C046C046C046C0460C4C4A
:102410001568246825605B08EAE765462C60146847
:102420003460F8E781F31088F0BDC046080500501D
:10243000080000200C05005000060020FC050020CC
:10244000F805002030B585B001AD0C220649280002
:1024500006F0E4FB0024285D01210134FFF730FD84
:102460000C2CF8D105B030BDBCA50000F0B585B08E
:102470006A463C4B3C4913801C2301AF93700C31DE
:102480000922380006F0CAFBFFF70CFD374B384D28
:10249000C0182B68984201D200232B602C68002CB6
:1024A00044D13E5D01213000FFF70AFD01340121D6
:1024B000300003F019FA092CF3D100246B461E5D9D
:1024C00001213000FFF7FCFC01340021300003F053
:1024D0000BFA032CF2D1C82080000138C046C04658
:1024E000C046C046C046C046C046C046C046C046BC
:1024F000C046C046F1D100210420FFF7E1FC6B4645
:1025000000211878FFF7DCFC6B4600215878FFF7B4
:10251000D7FC6B4600219878FFF7D2FCFFF7C2FC8E
:10252000002413302860200005B0F0BDFFF7BAFC8E
:102530002B6800249842F6D3042003F065F80D4B75
:102540000D4EC0180BD430603068032104F04EFDEE
:1025500000230A4A30602B6013600124E3E73460F3
:10256000F2E7C0461A1B0000BCA5000010270000BF
:10257000EC050020C8FEFFFFE0050020F405002068
:1025800010B50124044002D04410200010BD0D20DD
:10259000FDF7A0FFF9E700000022054B10B51A6017
:1025A000044B1B68934201D002F0DAFA002010BD00
:1025B000F0050020C410002070B508680D00FFF77A
:1025C000DFFF04006868FFF7DBFF621E0100042ADA
:1025D00014D8451E042D11D805236B439B180122E6
:1025E00015009D402B00064805682B430360054BF2
:1025F0001B68002B02D0200002F0B3FA002070BD4F
:10260000F0050020C410002070B508680D00FFF729
:10261000B7FF04006868FFF7B3FF621E0100042AD9
:1026200013D8451E042D10D805236B439B18012297
:102630009A400748036893430360064B1B68002BCE
:1026400003D00022200002F08CFA002070BDC046AA
:10265000F0050020C4100020F0B5050089B008681E
:102660000C00FFF78DFF0690022D36DD6068FFF746
:1026700087FF0190A068FFF783FF04000127231D57
:10268000661E0793731C0293079B9E4235D0052359
:1026900073430593019B019D05330493049BAB4257
:1026A0001ED0042E16D86B1E042B13D80122059BB6
:1026B0002349013B5B199A409446224A0B681068F3
:1026C000069A3A4003920DD062461A430A600122EC
:1026D00000280DD17F000135E0E701240194CDE70A
:1026E000029ECFE7624693430B600028F2D0039A24
:1026F0000299280002F035FAECE7019B1E1D042E1A
:102700001AD8012C18D1002505273B0021006B4366
:102710009B1999400B000A4A013511689943094BEE
:1027200011601B68002B05D0019B0022581D290059
:1027300002F017FA052DE8D1002009B0F0BDC0461F
:10274000F0050020C410002010B5041E10DA00248B
:102750000A4BA400E25801239340094A0949136037
:10276000094A1160094A0A4911600A4A136010BDFA
:10277000FFF7A4FBA042EADDEAE7C04640B2000052
:10278000FC0500200805005000060020F805002088
:102790000C050050180500500200086810B5C3076A
:1027A0000DD540101823012A03DD4A68042A00D100
:1027B0000833044A1360FFF7C7FF002010BD012053
:1027C0004042EFE7080000202B4BF7B51B680C00D8
:1027D000002B03D101204042FFF7B6FF01262468F9
:1027E00034421AD0FF226310120260121040DAB293
:1027F0001043FF221B021204134018431F4B1B6897
:10280000202B06D1B4401E4BA40EA400E3580002B6
:102810001843FFF7DDFD0020FEBD03252540FAD15A
:10282000042CF8D90F2322681340062BF3D1FF277D
:10283000130901933F02019B9D42ECDA0135AB0085
:10284000E3583342F7D05A105812D1B238400843F7
:10285000FF21120209040A401043084A1268202A84
:1028600006D15B009B0E06499B000202585810439C
:10287000FFF7AEFDDFE7C046FC05002008000020A2
:10288000ACA70000086810B5C30703D5FFF778FEB2
:10289000054B1860054B1B68002B03D0024B1868D2
:1028A00002F060F9002010BDF0050020C4100020E7
:1028B0000868F8B5C3071AD5FFF762FE0300203B8E
:1028C0005E2B25D80520012258430023114E451DBB
:1028D000A84219D005211024375C3C4200D09B1837
:1028E0000139520064100029F7D10130F0E7830765
:1028F0000ED104280CD90F2203681A40042A07D1EC
:102900001B0905D00079D9E701205B001843F8BD09
:102910000120FCE7D1A500007FB5A04C2368002B67
:102920000AD19F4A1268002A06D19E4B1B68002BD1
:1029300001D0FFF79BFD7FBD9B4D2A68002A26D161
:10294000984A1268002A1BD0FFF790FD0028F2D0A9
:10295000FFF778FD924B24681A681C60002A16D095
:10296000002C14D101AD0C229049280006F056F934
:10297000285D00210134FFF7A3FA0C2CF8D1DAE727
:10298000874A1268002AE5D1002BE3D0E0E7002156
:102990001A2002F0A9FF00211B2002F0A5FF002150
:1029A0001C2002F0A1FF2E68012E5CD0022E00D167
:1029B000A2E0002E50D101363100794C032023686B
:1029C000994302F091FF0420216801404B42594194
:1029D00002F08AFF102123680A2019404B42594116
:1029E00002F082FF80212368090119404B425941BE
:1029F000062002F079FF80212368090219404B422A
:102A00005941072002F070FF8021236849021940D4
:102A10004B425941092002F067FF80212368890257
:102A200019404B425941192002F05EFF8021236872
:102A3000C90219404B425941182002F055FF80232A
:102A400021681B0319404B425941172002F04CFFEB
:102A500031001A2002F048FF2B680321581C04F0B3
:102A6000ABFB296067E702214D4C17202368194012
:102A70004B42594102F038FF0821236818201940C1
:102A80004B42594102F030FF80212368C9001940B0
:102A90004B425941042002F027FF8021236849015D
:102AA00019404B4259410A2002F01EFF8021236841
:102AB000C90119404B425941032002F015FF802102
:102AC0002368890319404B425941092002F00CFF49
:102AD000802321681B0419404B425941192002F000
:102AE00003FF3100062002F0FFFE3100072002F054
:102AF000FBFE31001B20ADE72021294C1720236865
:102B000019404B42594102F0EFFE40212368182042
:102B100019404B42594102F0E7FE802123681920F9
:102B200019404B42594102F0DFFE802123684900E1
:102B300019404B425941092002F0D6FE80212368FA
:102B4000890019404B425941072002F0CDFE8021F7
:102B50002368890119404B425941062002F0C4FE06
:102B600080212368490319404B4259410A2002F051
:102B7000BBFE80212368C90319404B425941032001
:102B800002F0B2FE802321685B0419404B42594198
:102B9000042002F0A9FE01211C205BE7F0050020C3
:102BA000E8050020F4050020E4050020BCA5000095
:102BB000012010B54042FFF7C7FD10BD10B5034A14
:102BC0000921034800F080FF10BDC046ACA80000FA
:102BD000F4A8000030B502248025094B094AED0015
:102BE0009C505C59002CFCD0A124E400884202D304
:102BF0000021995030BD8025ED0018514019F5E7AE
:102C000000E001400405000010B5002806D1C020F6
:102C1000B02140028902FFF7DDFF10BDB020802106
:102C20008002C902F7E7000043425841064B404288
:102C30001840B0239B02C018036800201A0E532AC4
:102C400001D11B02180A704700C0FEFF30B50124F5
:102C50008025054B054AED009C505C59002CFCD0AA
:102C600001600021995030BD00E0014004050000E2
:102C700043425841074B40421840B0239B02C018C2
:102C8000A62310B50902DB05090A1943FFF7DEFF89
:102C900010BDC04600C0FEFF70B5012480250D4B5D
:102CA0000D4EED009C515C59002CFCD0002902DC3B
:102CB00000229A5170BD557814782D0225439478DE
:102CC000013924042543D478043224062C4310C04F
:102CD000ECE7C04600E001400405000070B50500C7
:102CE0004B680A009C1C2100A400FFF7D5FF28199F
:102CF00070BD0000134B1B68002B0CD08022B0234A
:102D0000D2029B0200280BD11A1D5B681B0E522BAE
:102D100000D110007047B022C02392025B02F1E79D
:102D200082420DD903681B0E522B09D1436802332E
:102D30009B00C018824203D903681B0E522BE9D0B6
:102D40000020E7E70407002070B50020FFF7D2FF5E
:102D5000FF260500002801D1280070BD03681C145F
:102D60003440FFF7C7FFDA2CF4D10500F2E700008A
:102D70008022F0B55200A1B00021674805F057FF4E
:102D8000802200215200654805F051FF644BFF2767
:102D90001B681A00049353425A4110000592FFF732
:102DA00033FF049C0020631E9C415E4B64421C4028
:102DB0005D4BE418FFF7C8FF0600002E2DD10498E4
:102DC000FFF732FF411C0598FFF752FF059A574D58
:102DD000534B2C601A60FFF79DF9514B64201B6820
:102DE000A0215A4253414F4A5B421340B0222C6803
:102DF00092029B18E41A6043490204F0F7F8A022FB
:102E00005202030000924A49220007A806F0EAFA9B
:102E100007A801F043F821B0F0BD32681314121274
:102E20003A403B4003921A000A3A092A49D83A4BE1
:102E3000039A995C002931D110223E4805F0F7FE33
:102E400035002B6803991A123A40914209D11A149D
:102E50003A400B2A27D0132A2DD00A2A01D1354B0C
:102E60001D602800FFF746FF051EEAD1314B1968A7
:102E700000290FD02000FFF731FF04002D4B5B1914
:102E80005968002903D02000FFF728FF040004350B
:102E90000C2DF3D1204B0121039A99543000FFF7F8
:102EA00029FF060089E73B40022BDADC214A9B0020
:102EB000D3185D60D5E7102200211E4805F0B7FE4B
:102EC000CFE71A00153A082AE8D8144A0399525C49
:102ED000002AE3D13500152B00D01500300003681F
:102EE0001A143A40152A0FD01D2A00D10025FFF7E9
:102EF00001FF0028F3D1002D04D020002900FFF7A6
:102F0000EDFE0400054BC6E7039A1B123B409A42B4
:102F1000EDD10500EBE7C046040600200C070020B9
:102F20000407002000C0FEFF04C0020008070020C4
:102F30008DA9000000250020F0B50020B7B00024C6
:102F4000FFF7D8FE270005002600002D2ED1284DC2
:102F50002868FFF769FE32003B0001900094254984
:102F600004A806F03FFA04A800F098FF224B642062
:102F70001C682B68A0215A425341204A5B421340EF
:102F8000B02292029B18E41A6043490204F02EF822
:102F9000A0225202030000921949220004A806F060
:102FA00021FA04A800F07AFF37B0F0BDFF226B6869
:102FB00029689C460233FF180B12013613409C42CD
:102FC00000DA1C00FF200A1402400392624601400E
:102FD00001920091039A0B4904A806F003FA04A891
:102FE00000F05CFF2800FFF785FE0500ADE7C04656
:102FF00004070020FEA900000807002000C0FEFF13
:10300000A8A90000EAA9000070B50020FFF70CFE97
:1030100004000120FFF708FE844200DA04000A4B96
:103020001D686A42554128001D60FFF7EDFDA02292
:103030006B4252021340054A28009B18044A611C47
:103040001360FFF715FE70BD040700200480010027
:1030500008070020F8B50020FFF7E6FD0700012073
:10306000FFF7E2FD3E00204D0643204C0DD18021AC
:10307000C020C9024002FFF7ADFD01213000FFF77B
:10308000F7FD1B4B2E6023601DE0874209DD002306
:10309000B0212B60164B8902236023680020012594
:1030A00017E0012380212B60124BC9022360F4E753
:1030B000120E522A08D0002800D023600E4800F0DB
:1030C000EDFEFFF7A1FFF8BD28005A68023292001A
:1030D0009B188B4205D21A68561CE9D10028F2D001
:1030E000D1E72160EFE7C046040700200807002071
:1030F0000480010004C00200C3A90000F0B585B03F
:10310000039203220333DC17294D1440E4182B6883
:10311000284F5A42534180225B42D202A4103B40C6
:103120009B18A21C0291244E9100009101903168DD
:1031300000980A18934215D2FFF71AFE2B685A42DC
:10314000534180225B421F40D202BF183368009A6D
:103150009B189F4206D2194800F0A0FE00252800C7
:1031600005B0F0BD029B356819066B461A7BA42397
:10317000DB051343FF222F00090C1943019B1204A6
:103180001B04134019432800FFF760FD0837281D72
:1031900021003760FFF75AFD002C04D00A9A210065
:1031A0003800FFF779FD009B083BFF183760D6E732
:1031B0000407002000C0FEFF0807002067A90000E8
:1031C00010B5FFF7D5FD10BD70B59AB0FFF742FFFF
:1031D000FF22254CD2000021200005F028FD002010
:1031E000FEF726FF04280ED10020FEF735FF042845
:1031F00009D1FFF709FF1D4800F050FE1C4800F000
:103200004DFE1AB070BDFFF79FFDFF250026002878
:103210000ED10200C300E3580130591E8B41D21871
:10322000FF28F7D1134901A806F0DCF801A8E3E76D
:1032300003681A142A400A2A0AD11A122A40FF2ABD
:1032400003D0D200A1180B71A050FFF753FDDEE7A9
:10325000132AFAD11B122B40FF2BF6D0DB00E21809
:103260001671E650F1E7C046781B002033AA000033
:1032700043AA00004BAA00000021094B094A5960EB
:103280000131516059680029FCD0002119610123E6
:1032900093600222044B8131FF315A501A6070470B
:1032A000FC1000400010004000E100E00222064B4C
:1032B0000121DA670022054B5A61054A11615A69FA
:1032C000002AFCD07047C04604E100E0FC1000403A
:1032D0000010004010B5044C2378002B01D0FFF7FC
:1032E000E5FF0020207010BD0D0800200120024BDA
:1032F0001B685B0018437047900800200348036870
:10330000002B02D11422037102607047282500208F
:103310000120024B1B685B00184370470C00002023
:1033200070B504000D001600FEF7BCFD80230122DD
:1033300000215B055B6E6270E270020AA271020CF2
:10334000E2711A0A60716372000EA2721A0C1B0EEF
:1033500026702571A1702072E272237370BD000087
:10336000124B10B51B68124C5A1C0FD0114C002B7D
:103370000CD0114C012B09D0104C022B06D00D4C57
:10338000042B03D00E4C052B00D10B4C21000D4813
:1033900006F052F8200006F057F803000422043328
:1033A0009B0809481B011343036010BD1000002057
:1033B000DFAA0000D8AA0000EAAA0000EFAA0000D5
:1033C000E4AA0000142500201025002070B5214C2F
:1033D0002278002A3DD1204B01215A608022D2055B
:1033E00011605A68002AFCD0002207201B4B1C49A0
:1033F00001255A500439585008315A5019481A4971
:1034000058501A491A485A501A495A50A622D200FE
:103410009D50082218495A5004315850022017492B
:103420005850174917485850174804395850182011
:1034300016495850C12189005A500539FF3958584A
:10344000921802435A501249124A9950FFF714FF3A
:10345000257070BD0D080020FC00004000100040E9
:103460000C050000746962751C050000240500004D
:10347000200004022C0500001405000034050000A3
:103480003C050000FFFF0000211001005405000072
:103490000E0800200405000070B50E4B06001B78D6
:1034A000002B01D1FFF792FF00200B4D2C788442B6
:1034B0000ED00A4B202219780323091B1940084B10
:1034C0004901C918300005F0A9FB0120013C2C700E
:1034D00070BDC0460D080020940800200C08002094
:1034E0000E080020002330B589B0984225DD032462
:1034F0000D682C409C4220D12300042D1DD90F21A2
:103500002A681140062918D112091F2A15D96846C0
:10351000FFF7C2FF230000280FD06B460122187866
:103520001300A04203DB6B461B5D5B0013430134B9
:10353000A1006B50202CF3D10423180009B030BD3A
:1035400070B5414B8AB01B78002B01D1FFF73EFFCD
:1035500002AD2800FFF7A0FF002802D100200AB02A
:1035600070BD2B780B2BF9D96B78012BF6D1EB784A
:10357000012BF3D10023354E354C336023712B7969
:10358000344A1360002B0ED1152169444A780B7818
:1035900012021A438B781B041A43CB781B06134381
:1035A0003360002318E0012B20D1152169444A78AB
:1035B0000B7812021A438B781B041A43CB781A211A
:1035C0001B06134333600E236A7C6944934200DD7B
:1035D000130000229A4232D104200021E218043361
:1035E0009B101B01034311712360B8E7022B03D129
:1035F0006A7B10331621E8E7042B0DD11521082230
:103600006944684605F00AFB0098019902F0DEF96A
:1036100005F0A8F93060C4E7052BC2D115210822B6
:103620006944684605F0FAFA0098019902F0CEF96B
:1036300005F098F930606A7D0A231E21C5E78D5C8C
:10364000A01805710132C5E70D0800209008002080
:10365000282500201000002010B5134B04001B7813
:10366000002B01D1FFF7B2FEFFF720FE00200F4A2A
:103670000F49104B545058600130106058680028B2
:10368000FCD0002018610130906018690028FCD03F
:10369000094B0A481B785B011B185350FFF706FEC5
:1036A000FFF7EAFD10BDC0460D08002000100040E5
:1036B00004050000FC1000400C0800200E0800204B
:1036C00030B589B000281EDD03230A6813401AD1E3
:1036D000042A18D90F2011680840062813D10909B7
:1036E0001F2910D90124013399005158002021428B
:1036F00001D04910C8B26D46591E6854202BF2D132
:103700006846FFF7A9FF002009B030BD10B50028BA
:1037100013DD0C68E30710D56410532C0DD8084B4B
:103720001B78002B01D1FFF751FEFFF7BFFDA1234E
:10373000044ADB00D450FFF79FFD002010BDC046B7
:103740000D0800200010004010B500280EDD0C68A8
:10375000E3070BD56410FF2C08D8054B1B78002B12
:1037600001D1FFF733FE034A034BD450002010BDB4
:103770000D080020001000402405000013B50028AB
:1037800014DD0C68E30711D5094B64100093094B55
:103790000193072C0AD8084B1B78002B01D1FFF7A7
:1037A00015FE6B46054A1957054BD150002016BD32
:1037B000E2ECF0F4F8FC00040D08002000100040DA
:1037C0000C05000070B588B0002820DD03240868CF
:1037D00004401CD104281AD90F2302681340042B7B
:1037E00015D1FEF745FD060005F02EFE0500122856
:1037F00000D912252A0002210D326846FFF790FDFC
:103800006B465D73A54205DC6846FFF725FF002087
:1038100008B070BD2300325D6B449A730134F1E748
:10382000F0B50D008BB0012831DD03240868044099
:103830002DD104282BD90F2302681340042B26D145
:103840004B68DB0723D5FEF713FD6E680700731086
:10385000019305F0F9FD05000E2800D90E252A0078
:103860000121113202A8FFF75BFD6A46127902AB13
:103870005A7302AA73129373019B76141B0ED673AC
:1038800013745574A54205DC02A8FFF7E5FE00207D
:103890000BB0F0BD3A5D02A963189A740134F1E7E8
:1038A00030B589B0002814DD0C68E30711D510226B
:1038B00068460021FFF734FD6B466A4665105D736C
:1038C000684663122D0E64149373D4731574FFF756
:1038D000C3FE002009B030BD174B184A59680029B3
:1038E00003D00021596001319160196900291FD06E
:1038F000002018618023DB00D3581149012B18D117
:10390000A923DB00D3585B420B600E490B78032BD5
:1039100001D801330B7003200B490B7801330340AE
:103920000B700A495B015B180949535001239360EE
:1039300070470860FAE7C046FC10004000100040E5
:103940000C000020940800200C0800200E08002025
:103950000405000010B5034A0E21034800F0B4F836
:1039600010BDC04668AA00005FAA0000044A0549CD
:103970001368C85401339B059B0D13607047C04604
:10398000B00C0020B008002070B5114C114A23681B
:10399000834202DC0023236016E0155C411C2E00EC
:1039A000FA3E012E05D899420FDA555C013D1F2DD4
:1039B00001D90800ECE70100151A565C6E5401317C
:1039C0008B42FADC181A206070BD1570FAE7C04609
:1039D000BC100020BC0C002010B5FEF759FA064BB5
:1039E0001A68824201D900221A601B68C31A034870
:1039F00098428041404210BDAC080020204E00009B
:103A000010B5094C094A23681268934200D110BDD1
:103A1000074AD05CFEF776FB0028F8D02368013314
:103A20009B059B0D2360ECE7B40C0020B00C00203C
:103A3000B008002010B50400064B074A1B68126846
:103A40009B1ADB439B059B0DA34200DB10BDFFF7D8
:103A5000D7FFF1E7B00C0020B40C0020F7B505004B
:103A600056680191B000441C06301700FFF7E2FFD2
:103A7000FB20FFF77BFF1C20FFF778FFE8B2FFF782
:103A800075FFE0B22412FFF771FFE0B2FFF76EFF9F
:103A90006B461879FFF76AFF0025AE4200DCF7BDE0
:103AA000AB00FB189C680135E0B2FFF75FFF201206
:103AB000C0B2FFF75BFF2014C0B2FFF757FF200E24
:103AC000FFF754FFE9E7000070B5074E3368092B94
:103AD00008DC0C255D43054C0133285164196160F5
:103AE000A260336070BDC046B80C00204C25002099
:103AF000F0B587B002900C00012803DC1B20FCF716
:103B0000E9FC45E0244B08680093830709D10428A9
:103B100007D90F2302681340042B02D1FEF7A8FB3C
:103B200000901D4B60680193830709D1042807D9D1
:103B30000F2302681340042B02D1FEF799FB01907A
:103B40000027164B1B680493049BBB42D6DD0C2652
:103B50007E43134B0099F618306805F063FC051E90
:103B600005D17368B6680593059B9D4201DB01375B
:103B7000EAE730680199039605F054FC08360028FE
:103B800008D121000298039B083102385B689847EE
:103B900007B0F0BD0135E7E7BFA40000B80C002076
:103BA0004C25002010B5FFF709F8FEF76BFAFEF779
:103BB000BFFBFEF7F5FBFFF7CDFE00F013FE00F0B4
:103BC000D3FF10BD962210B512010021034805F065
:103BD0002EF80022024B1A6010BDC04618120020B9
:103BE000B0050020064B074A1B6812689B1ADB438E
:103BF0009B059B0D0122834200DC002210007047D0
:103C0000B00C0020B40C0020F8B505000C00160024
:103C10001F1E0ED10320FFF7E5FF002808D0FA2071
:103C2000FFF7A4FEE8B2FFF7A1FEE0B2FFF79EFEA9
:103C3000F8BD501DFFF7D6FF0028F9D0FB20FFF795
:103C400095FEE8B2FFF792FEE0B2FFF78FFEF0B20A
:103C5000FFF78CFE3012C0B2FFF788FE3C00E31B7A
:103C60009E42E5DD2078FFF781FE0134F7E7000092
:103C700070B50024F0250B4B1B68A34202DCFFF754
:103C8000A1FF70BD2B006343074A9B181A78002AD6
:103C900005D05978002311201A00FFF7B5FF013431
:103CA000E9E7C046B005002018120020F8B507006B
:103CB0000024F0252B0063430C4A01349E18B742C0
:103CC00011D0317800290BD00133D15C00231120B1
:103CD0001A00FFF799FF2A000021300004F0A7FF27
:103CE0000A2CE7D1F8BD024B1C60F9E7181200203E
:103CF000B0050020F3B50400100001220300FFB05E
:103D00000D00134013D002AB1A70431002AA02A98F
:103D1000537042121B0E8A700B7105220B00401467
:103D2000C87029002000FFF76FFF7FB0F3BD0326A6
:103D300006401ED104281CD90F2201680A40042A1B
:103D400029D1022302AA1370FEF792FA070005F0A8
:103D50007BFBF823FF33984200D91800B04202DC05
:103D6000421C02ABDDE70136731EFB5C02AA9355D1
:103D7000F4E7042801D0002809D1032302AA04385B
:103D800013704242504102AB58700222C9E7002E24
:103D9000CBD10428C9D90F2102681140052913D1BC
:103DA000013902AE3170F8211209FF3192008A42C6
:103DB00000DD0A00934201DB0132D2E70133C11872
:103DC000C97802AEF154F5E70629AED101390E00EB
:103DD000120956430196F826019FFF36B742A4DC2C
:103DE00002AE31700136934201DB019AE4E701270C
:103DF00001339900415839420BD0394101273770BE
:103E00000F127170B7700F14090EF770317105360B
:103E1000E9E70149F2E7C04619FCFFFF70B502006F
:103E20000024F0210D4E080060438019457895422A
:103E300003D001340A2CF6D170BDF022002104F029
:103E4000F6FE074A1368013BA34200D11460002329
:103E500029001A001120FFF7D7FEEDE71812002005
:103E6000B005002010B5B2B002236A4604001370FA
:103E700005F0EAFAC72800D9C7200023984207DCDA
:103E8000421C6B46FE211420FFF7BEFE32B010BD6F
:103E9000694601335A1EA25CCA54EFE730B5B3B08D
:103EA00002236A460500137005F0CEFA0400C72805
:103EB00000D9C72400239C420BDC20003230FFF7DE
:103EC000B9FD621C6B46FF211420FFF79DFE33B045
:103ED00030BD694601335A1EAA5CCA54EBE70000A4
:103EE000F7B5234B06001B68F02100930023009ACE
:103EF0009A4211DC0024F0231A00624301920199D6
:103F00001C4A55182F78002F12D001340A2CF3D1F7
:103F10001948FFF7C3FF29E00A005A4315488218E1
:103F20005078B04202D11278002A1FD10133DEE767
:103F3000F0223900280004F07AFE02230D4A01998C
:103F4000EB6053540D4AF1008A58009B6E70AE70BE
:103F5000AA602F616F61A34202DC054B01341C6033
:103F6000002331001A001020FFF74EFEF7BDC046B7
:103F7000B005002018120020D9AF0000781B0020E7
:103F800010B5FFF775FEFF24084AE3005B429B185B
:103F9000074AD35C043B012B03D8E043C0B2FFF7D0
:103FA0009FFF013C002CEFD110BDC046FC07000074
:103FB000781B0020F7B50E00FF247F2501901C4AD6
:103FC000E300D31A1B4A9A181278062A01D0032A52
:103FD0001DD1FF22D2009B18186883682B401C2B30
:103FE00015D1C3681A002A40042A10D102692A4058
:103FF000192A0CD11B0A01339B000C30C018FEF7A4
:1040000037F9070005F020FA0023B04209D0013C3F
:10401000002CD4D1F7BD019AF95CD25C9142F6D163
:1040200001339E42F7DCE043C0B2FFF759FFEEE7F1
:10403000781B0020FC07000070B50500FF24084A2B
:10404000E3005B429B18074AD35CAB4203D1E043D9
:10405000C0B2FFF745FF013C002CF0D170BDC04657
:10406000FC070000781B0020F7B5FDF711FF514B4E
:104070001A68824201D900221A601A684E49821ACF
:104080008A4200D883E01860FDF70CFF071E00D1BC
:1040900001370020FDF7CCFF01900020FDF7DCFF89
:1040A000019B0090454C464D002B14D02368002BFB
:1040B00000D07AE02B682760002B00D171E0414BE3
:1040C00001261B78002B63D10920FFF7B5FF3E4B7B
:1040D0001E703C4B1E70009B002B12D02B68002BD7
:1040E0000FD123682F60002B1ED0374B01261B7881
:1040F000002B52D10920FFF79FFF334B1E70314B2D
:104100001E702368002B0FD02F4E3278002A0BD15F
:104110009F4200D227602368FB1A312B04D9072065
:10412000FFF78AFF012333702B68002B0FD0254E39
:104130003278002A0BD1BB4200D92F602B68FF1ABE
:10414000312F04D90820FFF777FF0123337023684C
:10415000002B0CD0019B002B09D11B4E3378002B78
:1041600002D10720FFF768FF0023236033702B681C
:10417000002B0CD0009B002B09D1124C2378002B74
:1041800002D10820FFF758FF00232B602370F7BDF2
:104190000720FFF751FF0C4B9CE70820FFF74CFF6F
:1041A000ADE7009B002B9CD1ABE7009A002A95D18C
:1041B000AAE7C046A80800200F27000098080020A2
:1041C000A0080020A40800209C08002037B5002487
:1041D0000500FFF74DFD01A80194FDF717FF210031
:1041E0002000FEF7D9F9FEF797FBFDF749FFFDF731
:1041F00048FFFEF7DDFCFDF771FEA54204D0FDF798
:1042000097FF0248FFF74AFE37BDC046CAAF00001D
:10421000002310B501001A001120FFF7F5FC10BDB6
:1042200007B56B46197069465A7013128B701314D8
:10423000120ECB700A716B46010005221320FFF7A6
:10424000E3FC07BD10B50A0001001220FFF752FD84
:1042500010BD70B5050008000C003230FFF7EAFB16
:104260002B00220000211B20FFF7CEFC70BD10B5F3
:104270000C000300110014202200FFF7C5FC10BD44
:10428000012370B5FF24084A41185B42884201D3DC
:10429000D84370BD06781D0A234073409B009B588D
:1042A00001306B40F2E7C046ACAB0000002313B511
:1042B00001930B4BC2000400D058002805D043687E
:1042C00008309900FFF7DCFF01900920FFF7B2FBEF
:1042D00001AB042221001720FFF796FC13BDC04656
:1042E000781B002070B506000020FEF703FD0024B7
:1042F000FF25002801D1200070BD03681A142A4050
:10430000152A07D11B122B40B34200D10400FEF73F
:10431000F1FCEEE71D2AFAD10024F8E7F0B580277A
:104320009DB0FFF76DFBAD4CAD4D2068FF00391A15
:104330004019FDF7CDFE23680600C3182360002B4B
:104340000ED11DB0F0BD2068391A2818FDF7C0FE47
:10435000236806001B182360FDF79AFDA14B186027
:10436000002EF0DC2B78FA2B00D013E12368022B0F
:1043700007DCFFF731FB0028E3D00120FFF704FB47
:10438000DFE76878AC78023818281FD802F09AFD69
:104390000D2024282B341E3E6872768CDEEF1E1E04
:1043A0001E1E1E1E1E1E1E1EFD00FF2C0ED02000F7
:1043B000FFF734FD00228C4BE100CA505B181A71E4
:1043C0002100009213001320FEF798FE0320D5E78A
:1043D0002000FFF785FDF9E72000FFF71FFDF5E757
:1043E000FFF7CEFDF2E7FFF743FC0020FFF7EEFEFC
:1043F0007E48FFF753FDE9E7632CE7D87C4BA2002A
:10440000D25821001520FFF775FCDFE700242000BB
:10441000FFF768FF061E03D10134642CF7D1D5E7FE
:10442000083005F011F805000530FFF703FBFB200D
:10443000FFF79CFA1D20FFF799FAE0B2FFF796FA12
:10444000E8B2FFF793FA2812C0B2FFF78FFA3700ED
:10445000BB1B9D42E0DD387AFFF788FA0137F7E7AA
:1044600000211D2000910B000A00FEF747FEFDF71A
:104470005FFEABE72000FFF719FFA7E7FDF71AFD86
:1044800003AC5C4A642100905B4B200004F078FF91
:1044900002232000237004F0D7FF23000200002134
:1044A0001620FFF7B1FB91E700244F4AE300D558EF
:1044B000002D28D06B689E00701DFFF7BBFA2B0003
:1044C00000253200083321000120FFF79DFB00206A
:1044D000FEF710FC2F002E00002818D1002F04D06A
:1044E0003A0001212000FFF7B9FA002D04D02A007C
:1044F00002212000FFF7B2FA002E04D03200002182
:104500002000FFF7ABFA0134FF2CCED15EE7FF218C
:1045100003681A120A40A24209D11A140A400B2A4F
:1045200008D10B400CD0012B0CD0022B0CD0FEF785
:10453000E1FBD1E7132AFAD100252F002E00F6E780
:104540000600F4E70700F2E70500F0E70024FFF7B4
:104550008FFB2200210000942300DA20FEF7CEFD1D
:10456000FF222100D200204804F061FB7FE7012CEC
:1045700002D1FEF7E1FC29E7022C02D1FEF720FE72
:1045800024E70120FFF722FE20E7002321001A0084
:104590001A2086E7FB2B00D0EFE62268042A00DC15
:1045A000E7E62E79E878154B360206439E4200DD99
:1045B000E3E6331D9A4200DCDBE6EB5CFE2B00D029
:1045C000DBE66B78AC78711E1B2B6BD018D8012BF7
:1045D0002BD0082B3DD0701DD0E6C046BC1000206B
:1045E000BC0C0020AC080020781B0020ACAF000001
:1045F00070230020C3AF0000BEAF0000F603000030
:104600001D2B60D052D31E2BE5D1012CE3D1002904
:10461000E1DD6B79002B03D01C00322B00DD32244E
:1046200064235C43344B1C60D5E7FF2CD3D02000BF
:10463000FFF7F4FB6D79314AB31E009221002A0086
:104640000A20FEF75BFD2E4BE400E0501B191D71A4
:10465000C1E7632CBFD86A79022A13D0032A1BD082
:10466000012AB8D1E979AB79090219432B7AA40060
:104670001B0419436B7A1B060B435B001343214A4F
:10468000A350A8E70029A6DDB11E1C48FDF7D4FD04
:104690001C4BA400E0509EE7AB79A4005A1E934146
:1046A0009B00ECE71848FFF785FC94E7FF2C92D0BD
:1046B0006A79022A8FD811490B2000912100B31E7C
:1046C000FEF71CFD87E70B00632900DD6323002252
:1046D00003A893420ADCD9430022C91719404118A4
:1046E0000A700133009021001520E9E7A9184979E3
:1046F00081540132EDE7C04604000020C20C0020C6
:10470000781B002070230020C10C00200122094BDF
:104710001A60094A1368002BFCD00322074B1B6860
:10472000D8171040C01801238010063840001843E5
:104730007047C04600C0004000C1004008C50040AE
:104740000120704710B5064C200000F045FB0549DC
:10475000200000F069FB0122034B1A6010BDC04627
:10476000E8100020801A0600C010002010B50121BA
:104770000D20FDF7A5FB01210E20FDF7A1FB002177
:104780000F20FDF79DFB044C200000F061FA102182
:10479000200000F079FA10BDC810002010B50468A0
:1047A0000D20E30703D56410FF2C03D91720FBF776
:1047B00091FE10BDFFF7DAFFE1B2024800F086FA81
:1047C0000020F6E7C810002010B5FFF7CFFF00214A
:1047D000034800F07BFA43000120184310BDC04697
:1047E000C810002010B5034A07210348FFF76CF9F1
:1047F00010BDC046F0AF000028B000000D4B70B5F2
:104800001B6804000E001500002B01D1FFF79AFF72
:10481000E1B2094C200000F09EFBF1B2200000F054
:10482000A1FAE9B2200000F09DFA200000F0FEFBA2
:1048300070BDC046C0100020E810002010B5012453
:104840000368234205D04168214202D08268224297
:1048500003D10D20FBF73EFE10BD5810802801D972
:104860001520F7E74910FF2901D91620F2E7521069
:10487000FF2A01D91720EDE7FFF7C0FF0020EBE783
:10488000F7B501242300A0421BDD0D682C4218D08F
:104890001A4B25411B684C68002B01D1FFF752FFD2
:1048A0000127174EE9B2300000F055FB3C420AD018
:1048B0003C413000E1B200F055FA300000F0B6FBA8
:1048C00000231800FEBD03252540F6D1042CF4D9A1
:1048D0000F2322681340062BEFD113090193019B8C
:1048E0009D42EADA0135AB00E1583942F7D0491070
:1048F000C9B2300000F036FAF1E7C046C01000201F
:10490000E8100020144B70B51B6805000E00002B4A
:1049100001D1FFF717FF114CEDB22900200000F084
:104920001AFBF1B2200000F01DFA0021200000F077
:104930001DFB002801D0404270BD0122290020004B
:1049400000F004FB200000F0FEF90028FAD020005F
:1049500000F0FEF9F0E7C046C0100020E81000208B
:1049600010B501240368234202D04168214203D1DB
:104970000D20FBF7AFFD10BD5810802801D9152080
:10498000F7E74910FF2901D91620F2E7FFF7BAFF30
:1049900040002043EFE70000002370B5344D0400D1
:1049A000EB5601330BD10D211D20FFF7ABFF5A2829
:1049B00014D101222A212A703D38FFF71FFF00235E
:1049C000EB56022B2AD0032B49D0012B4CD12100CE
:1049D0001D200124FFF796FF644225E00F211920D6
:1049E000FFF790FF332805D102235F222B7020218F
:1049F0001A38E2E70D211E20FFF784FFC7280AD1ED
:104A0000032300222A21A9382B70FFF7F7FE1B226F
:104A10002A211E20D1E700232B70D0E7012C13D1CF
:104A200029211920FFF76EFF7F2801DD0138FF38AB
:104A300003007F3301DA7F20404264237F21584303
:104A400002F0D4FA604370BD032C0BD12B21192046
:104A5000FFF758FF043CE7E72D211920B9E72100B3
:104A60001E20B6E7052CF7D0012400206442E4E7BD
:104A70001400002010B50120FFF78EFF4300012035
:104A8000184310BD10B50320FFF786FF4300012037
:104A9000184310BD10B50520FFF77EFF430001202D
:104AA000184310BDF8B50123020018009A4236DD04
:104AB0000E68334233D003244D682C402FD1042D8F
:104AC0002DD90F2229680A40062A28D1144B1B68C9
:104AD000002B01D1FFF736FEEB0704D42B681C092D
:104AE000202C00DD20247610F1B20E4E2200300082
:104AF00000F02CFA0435A700EF19AF420CD03000BB
:104B000000F021F90028FAD0300000F021F901234B
:104B10004000184301C5F0E7012064002043F8BDC0
:104B2000C0100020E81000200020704701207047CE
:104B30000020704700207047012070470020704718
:104B40000020704700207047002070470020704709
:104B500000207047002070470020704700207047F9
:104B6000704770477047000010B5034A0E21034894
:104B7000FEF7AAFF10BDC0466CB00000DCB000001C
:104B800010B5FDF78BFA0648FDF7F6FAFFF70AF8BD
:104B90000448FFF783F9FEF717FBFFF7F1F910BDA3
:104BA000E204000065B1000010B5FDF70BF910BD7F
:104BB00070B5002504AC24780573A94205D10A4BD1
:104BC0000A4A23210A4803F0ADFF01600949920017
:104BD00052589B0002715B58A40083716358856032
:104BE00043710223C37170BD7DB10000E2B10000CA
:104BF0008BB1000040B20000037B002B04D1437353
:104C00008373036101330373704700001FB5019183
:104C1000A02100240068C900D2B24450012A10D05B
:104C2000A24209D0032A0AD0074A8350074B019AAF
:104C3000C250012343501FBD02221343F4E7042254
:104C4000FBE70622F9E7C0465405000024050000F2
:104C500010B50400FFF7D0FFA1222368A179D2008C
:104C600099506179064A200099502179043299506F
:104C7000044B19685A689B68FFF7C8FF10BDC0460F
:104C80000C050000DC1000204BB2002B0FDB802352
:104C90003F290FD81F290FD80F290FD807290FD860
:104CA00003290FD81B060168074A8B5070478023E1
:104CB0009B04F8E7DB04F6E71B05F4E75B05F2E786
:104CC0009B05F0E7DB05EEE7240500000368074AD3
:104CD00099501A00FC32D1680029FCD0A321C900E8
:104CE00058580023C0B2D3607047C0461C0500006E
:104CF00007B58022074BD2051A6000229A60023263
:104D00001A710F230C3200930349023B0348FFF74B
:104D10004FFF07BDDC10002000300040C81000200D
:104D2000F8B505000E0017000024BC4208D02B681F
:104D3000315D1B6828009847002801D00134F4E752
:104D40002000F8BD704710B51C3000F0A9F910BD67
:104D500010B51C3000F096F910BD10B51C3000F0F5
:104D6000A5F910BD70B5437E0D00002B01D10020C8
:104D700070BD6430040000F0A2F90028F7D12000D3
:104D8000290000F070F90120F2E70000F7B5019367
:104D9000FA23002504009B0083600D4B4560083317
:104DA00003601C300F00160000F052F92000643040
:104DB00000F04EF9074A2761B600B358200063752A
:104DC000019B9B009B586576A576A375FEBDC046EA
:104DD00020B2000040B200000123A022C375837DF1
:104DE0000E49C133FF33D2059B009950437DC13337
:104DF000FF339B009950CC220169094B5204CA50E1
:104E000005220169243BCA50827D01690833CA50DA
:104E10000269417D034BD1507047C0460C0600002B
:104E2000240500000C050000A022002310B5046931
:104E3000D200A3500A4CA1420FD90A4C8C425B41CC
:104E400009495B420B40CD21C9045B18046907493D
:104E5000635005210369995010BDCC235B04F5E72D
:104E6000A086010090D00300000098FD24050000FA
:104E7000F7B5040000200D000193824265D01600B2
:104E8000402A00D9402627001C37380000F0F6F8E9
:104E9000B1232269DB00D5508022012321699200D1
:104EA0008B50A27E002A03D122691362226913600B
:104EB0000025731EAB4207D1019B002B04D080223A
:104EC0000221236992009950012223691A62236901
:104ED000FC33DA68002A02D19A6A002AF9D09A6A69
:104EE000002A0BD1DA60A3232269DB00D1583800F5
:104EF000C9B2013500F0B7F8B542DAD3019B226997
:104F0000002B0FD11300FC339B6A002B0AD1013315
:104F1000A376D3612369FC33DA6C002AFCD000222B
:104F2000DA640AE000230121A37651611A002369A3
:104F3000FC3399680029FCD09A602369FC339A6A93
:104F4000002A01D000229A62E8B2FEBD10B501230A
:104F5000FFF78EFF10BD0300AC3310B504001970CD
:104F6000643000F08BF80123637610BD002302004B
:104F700070B5AC3243760D001178B122040000699F
:104F8000D20081508022216992008B502269013326
:104F900013622269936026006436300000F080F8C6
:104FA000002812D0300000F06DF81E4B2269D0505E
:104FB0002369FC331A6A002A02D19A6A002AF9D0BE
:104FC0009A6A002A01D11A62E5E723690122002DBD
:104FD0000DD11900FC31896A002908D1DA612369F1
:104FE000FC33DA6C002AFCD00022DA6407E05A6154
:104FF0002369FC339A68002AFCD000229A600020C2
:105000002369FC339A6A82420BD098622169064A6E
:105010008B588B501800022B03D0181F431E984149
:10502000033070BD1C050000C404000010B5012150
:10503000FFF79CFF10BD000010B513231422024996
:105040000248FFF7A3FE10BD00400040E81000201A
:1050500010B540220021040003F0E9FD00232000E8
:105060002364636410BD10B53F24026C531C2340BD
:10507000446C9C4201D08154036410BD002303643E
:1050800043647047436C026C934206D03F21C25C7C
:1050900001330B4043641000704701204042FBE79E
:1050A000036C406C181A00D540307047436C026C9A
:1050B000934201D0C05C704701204042FBE73F2291
:1050C000036C406C01331340181A43425841C0B27C
:1050D0007047000003210A4802680A430260094839
:1050E00002680A4302600849084A094B9B1A03DD1B
:1050F000043BC858D050FBDC00F012F8FBF704F872
:1051000024050040540500404CB70000000000207A
:1051100048020020FEE7FEE7FEE7FEE7FEE7FEE7C7
:105120002D4B10B51A68D2B2012A0FD12B4A126842
:1051300012070BD12A4AE0241168F022080010401F
:1051400021422DD12749096811422CD01A68D2B2C8
:10515000012A12D12149096809070ED1F0202049FE
:1051600009680140402908D11E490968014204D15B
:105170008020C121C005C90042501B68DBB2012B51
:105180000DD1164B1B681B0709D1154B1A68F0236C
:105190001A40A02A0FD1134A12681A420ED010BD2D
:1051A0003028CFD0D2E7104A104911608021104A30
:1051B00009021160CAE7D02AF1D1ECE70D4B1A6859
:1051C000012A04D00C4A1A601A68012AFCD1C022B4
:1051D0000A4B1A60E3E7C046E00F00F0E40F00F06E
:1051E000E80F00F0EC0F00F004050040DFFF07C0FF
:1051F000186C004000EC06407593000014EC06406B
:105200000120704710B503681322DB69984710BD71
:1052100070470000054B0269D1500369FC331A6ADC
:10522000002AFCD0002201201A6270471C050000F1
:10523000030010B55C331A781F231A401E3B190077
:105240009140114AD167C222042104699200A15001
:10525000026953600269D360A02300220169DB0068
:10526000CA5001230169094A5B428B500169084A0F
:105270008B5001690C3A8B50016908328B50143005
:10528000FFF7FCFE10BDC04604E100E00C05000085
:105290001405000010B51430FFF702FF10BD10B563
:1052A0001430FFF703FF10BD10B51430FFF7EAFE0E
:1052B00010BD0000030070B55E331A780469724BAC
:1052C000E25003005D331A780469704BE25003002A
:1052D00061331C7802696E4B012C00D09EE0050002
:1052E0005F352E78A225ED00565102006032157808
:1052F000A1220669D200B5500269D4509623DB0082
:10530000994200D88CE096231B01994200D88AE08C
:1053100096235B01994200D888E096239B0199422D
:1053200000D885E0E1239B01994200D882E09623D2
:10533000DB01994200D880E0E123DB01994200D8EB
:105340007DE096231B02994200D87AE0E1231B02FC
:10535000994200D877E096235B02994200D874E026
:10536000E1235B02994200D871E0E1239B0299425C
:1053700000D86EE0474B994200D86CE0E123DB0295
:10538000994200D86AE0E122002312038A425B417D
:10539000414A5B421340802252059B1801693F4AF3
:1053A0008B50A02304220169DB00CA50002103694D
:1053B000FC33D9600369FC331962012301690B6076
:1053C00001698B60C1210469890062501F215C3032
:1053D00002780A4093406231314AFF315350002134
:1053E000415600293CDA0F230B40083B2D4C9B080B
:1053F0009B001B1903242140A140FC348C40DD6933
:10540000A5432C00C0258D4029002143D9611F23CD
:10541000017819401E3B8B40136070BD00246CE77F
:105420009E23DB02BAE79D231B03B7E71E4BB5E7BC
:105430001E4BB3E7EC239B03B0E71D4BAEE71D4BC0
:10544000ACE71D4BAAE71D4BA8E71D4BA6E71D4B7C
:10545000A4E71D4BA2E78023DB049FE71B4B9DE7DE
:105460008C080F4BA400E41803230B40FF21C02538
:10547000DB009940AD0066598E433100C0269E4046
:1054800033000B436351C2E70C0500001405000014
:105490006C05000090D0030000D0BEFE2405000083
:1054A00000E100E000ED00E000B013000050270034
:1054B00000A04E0000F0750000509D0000F0EB00D1
:1054C00000903A0100E0D70100B0AF0300705F0721
:1054D000F7B5009308AB1B7800250193FA2304006D
:1054E0009B0083600E4B45600833036014300F004F
:1054F0001600FFF7ADFD23005C3327611E70009B93
:10550000084A9B00995823005D331970019B2000C5
:105510009B009A5823005E33DD701A70FEBDC046B2
:10552000C4B2000040B20000036910B51A00FC329A
:10553000D2680400002A0AD0A322D200995814305D
:10554000C9B2FFF790FD00222369FC33DA6010BD79
:1055500010B50248FFF7E8FF10BDC046A0110020BB
:10556000162307B5022200930249013B0248FFF7C8
:10557000AFFF07BD00200040A011002070470000D1
:1055800010B500F011F8FFF7F9FF012000F000FA64
:10559000FFF7F6FAFFF708FB024B002BFAD000E00A
:1055A00000BFF7E700000000C420114B80001A582C
:1055B00010491140C02212020A431A50C021802211
:1055C000490092025A501A608023A3220021DB0571
:1055D000D20099500122F9309A60074BFF301950E0
:1055E000C120023180001950403019501A607047B4
:1055F00000E100E0FF00FFFF00100140014B1860D8
:105600007047C04660000020F7B5002320285AD814
:10561000384B8000C258042A5BD007D8022A54D0E5
:1056200055D80423012A09D000234CE0062A54D07F
:1056300051D31A2A53D002231B2AF5D12E4A1168BE
:1056400008294ED909294FD00A240226A020012575
:105650002A4AC00015502A482A4D07681C20BF005E
:1056600007402948019700685759009027481B02B6
:1056700007401F43C02300989B020340FF2057515F
:105680005759000207401F43019B1F43009B5801CD
:105690006023184007433E43565101251C4B1560BB
:1056A00058680028FCD000205860A1230125DB00A9
:1056B000D3585560A025ED0050511BB2A14202D035
:1056C00015D2611ACB401800FEBD0823B6E710239F
:1056D000B4E72023B2E74023B0E78023AEE70123FD
:1056E000ACE708240026B1E70C000126AEE7091B51
:1056F0008B40E8E740B200005C00002000700040F2
:1057000018000020040500001C000020FF00FFFF1F
:10571000FC700040F0B520285BD8364B8000C258A2
:10572000354B1E68002E30D1C227344BBF00D859EC
:10573000334C03250440C02000022043D851C0242C
:1057400080206400800018512E4F18602E4B803C42
:10575000D859FF3CA043D8510437D859A843204317
:10576000D8510837D8590C35A843844607206546D8
:105770002843D851A820C0001E50C1208026800098
:1057800076021E501C601C4B1C60142500202B0050
:105790001E4C2E0046433659771C1BD14343E25022
:1057A000A0230325C132FF329200DB05D550184BF0
:1057B0001A68082A14D114234343E3189A6812483C
:1057C0005132FF32920059601150DA68C1239B00B8
:1057D000C250F0BD9642E1D001300328D9D1F8E79C
:1057E000082A02D9083AD140E5E708239A1A9140DD
:1057F000E1E7C04640B200000412002000E100E0F2
:10580000FF00FFFF04050000009000402000002082
:10581000600000202149F0B54A6C2148002A14D0CC
:10582000A025A12600230124ED05F600C258571C2F
:1058300006D0C7187F68002F02D027009740AF51CD
:1058400014333C2BF2D100234B64A0230121DB0550
:1058500000260F009C4614234B43C3181A1F1268DE
:10586000104C0E4D920014195219526C002A10D08F
:105870001A00143A1268551C09D0103B1B68FF2B04
:1058800005D03B00934065461A00074BEA50FC34B4
:10589000666401310429DED1F0BDC046FC900040B1
:1058A00020000020009000400C05000000B52028DA
:1058B00010D80C4A8000835803290BD8A022080076
:1058C000C133FF33D2059B0001F0FCFA0209050742
:1058D0000021D15000BD0C21FBE70421F9E7032191
:1058E000F7E7C04640B2000020280AD8074B8000E6
:1058F000C25801239340A022D205002902D10449B5
:1059000053507047A121C900FAE7C04640B20000D9
:105910000C05000003000020202B0AD8A021A222A1
:10592000C905D2008858034A9B009B58D8400123E0
:105930001840704740B20000F7B506000D000C009B
:105940008B180193019B671B9C4207D03368217819
:105950001B683000984701340028F3D13800FEBDA1
:105960000849094A094B10B51B688858FA22190AD8
:105970001B0618439200002301F070FC4904C00B81
:10598000084310BD0010014004050000081200206B
:1059900070B5041E09D0FFF7E3FF050000F014F80E
:1059A000FFF7DEFF401BA042F8D370BD0022044B7E
:1059B0009A60044A13680133DBB213607047C04633
:1059C000FC1001400812002070470000F0B5C646E8
:1059D00000B5CB0F9846404A4B005B0D9A1882B039
:1059E0000D000400132A2FDC002A49DB3B4F17412E
:1059F0003E000E40064323D07F08390029400C4367
:105A00000AD03749BD438C4663445C425C418023E5
:105A1000DB021341E4071D434146CE0031492B0010
:105A20008E192200346875682000290001F0BCFD41
:105A3000009001910098019922002B0002F04AFC8D
:105A400002B004BC9046F0BD332A08DD8023DB00A1
:105A50009A42F5D102000B0001F0A6FDF0E7224AC0
:105A60009446012263445242DA400242E8D052088E
:105A70000242D1D094438022D2051A411443CBE78D
:105A80004B005B080343DBD00B031B0B1C4363423F
:105A9000234380244D0C24031B0B23406D042B4314
:105AA00019004346DA000F4B9B181C685D68020022
:105AB0000B002000290001F077FD00900191009873
:105AC000019922002B0002F005FC42464B005B08C6
:105AD000D60733431900B3E701FCFFFFFFFF0F00B8
:105AE000EEFBFFFFF8B20000EDFBFFFFF8B5274A21
:105AF0004B005B0D9A180C000700132A10DC002ADB
:105B000036DB234B13410B423AD08024240314414B
:105B1000002064189C430600250030002900F8BDD1
:105B2000332A0EDD80230600DB000D009A42F4D1FB
:105B300002000B003800210001F036FD06000D00C8
:105B4000EBE7144D0600AC46012563446D42DD4091
:105B5000AC4663460D000342DFD033239A1A323B32
:105B600093401818874200D94C1C63469843D2E7EB
:105B7000C90FCC070020531CCDD1074B1C43CAE7EB
:105B800006000D000028C0D1C7E7C04601FCFFFF9A
:105B9000FFFF0F00EDFBFFFF0000F03F30B5214A93
:105BA0004B0087B05B0893421EDD1F4A934205DD20
:105BB00002000B0002F08EFB07B030BD02AA00F01D
:105BC00035F803231840049A059B012813D00228B6
:105BD0001DD0002814D00298039900F037FA8023D2
:105BE0001B069C466144E7E7002300220093002344
:105BF00000F0A6FFE0E70298039900F027FADBE740
:105C0000012402980399009400F09AFFD4E701243C
:105C100002980399009400F093FF80231B069C4692
:105C20006144C9E7FB21E93FFFFFEF7FF0B54E4636
:105C30004546DE465746E0B5E14B4C008FB09046F6
:105C4000894664089C4200DC87E0DE4B9C4222DCF3
:105C5000DD4A002900DC92E0DC4B02F03BFBDB4B31
:105C600006000F009C4200D17EE1D94AD94B02F0D8
:105C700031FB02000B00414630000A604B603900E6
:105C800002F028FBD34BD24A02F024FB4346012505
:105C90009860D9606BE0D04B9C4200DC8FE0CF4B2A
:105CA0009C4200DD55E1CE4A231592469A44514666
:105CB0000905631A19001D00040002F053FE02F0EA
:105CC00087FE02000B00200029000892099302F0D1
:105CD00001FB0022C34B02F08BF80F00060002F01C
:105CE00041FE02F075FE04000D0002000B003000C2
:105CF00039000A940B9502F0EDFA0022B94B02F03C
:105D000077F8002200230C900D9101F079FA002819
:105D100000D192E1002300222000290001F070FA56
:105D2000434243410133B04A41460192022208A84E
:105D30000092524600F0A4FA4B460500002B16DAFA
:105D4000802243461206944642465B6845426344BD
:105D50005360D3686344D36009E00B0002004146FE
:105D60000A604B600022002300258A60CB60280077
:105D70000FB03CBC90469946A246AB46F0BD934B53
:105D800001F012FC914B06000F009C4200D13DE156
:105D90008F4A904B01F008FC02000B004146300096
:105DA0000A604B60390002F095FA894A894B01F08C
:105DB000FBFB012543466D429860D960D7E700F0B0
:105DC00071FF8A4A8A4B06000F0002F011F8002288
:105DD000884B01F0E9FB02F0C5FD050002F0F8FD7B
:105DE000794A7A4B0490059102F002F802000B0008
:105DF0003000390002F06EFA754A06000F00049870
:105E00000599744B01F0F4FF029003911F2D00DC03
:105E1000C7E0029A039B3000390002F05BFA834628
:105E20008A4653465B0024155B0DE31A102B6CDD8C
:105E300004980599D322674B520501F0D9FF02005F
:105E40000B00300039000292039302F043FA0A007B
:105E5000010013000691079202003900300002F0A1
:105E600039FA029A039B02F035FA06000F000498F3
:105E70000599614A614B01F0BBFF32003B0002F023
:105E800029FA069E079F0B0002003900300002929B
:105E9000039302F01FFA4B005B0D83468A46E41A17
:105EA000312C32DD04980599B822544B920501F04B
:105EB0009FFF03000C000200029303940B0006985E
:105EC000079902F007FA02000B0006000F0006987F
:105ED000079902F0FFF9029A039B02F0FBF9484A86
:105EE0000290039104980599464B01F081FF029AB4
:105EF000039B02F0EFF902000B0030003900029220
:105F0000039302F0E7F983468A465A4653464146D0
:105F100030000A604B60390002F0DCF9029A039B02
:105F200002F0D8F944460B000200A260E3604B4641
:105F3000002B00DB1BE75B46236080231B065344DA
:105F4000636080231B069C466144A060E1606D4253
:105F50000DE70B00020002F0BDF9434600259860F2
:105F6000D9601860596002E7D3221A4B520502F03B
:105F7000B1F9214A214B0D00040002F0ABF90200F7
:105F80000B00414620000A604B60290002F0A2F994
:105F90001A4B194A02F09EF9434601259860D960D0
:105FA000E5E602000B003000390002F093F96B1EA9
:105FB000154A9B009B5883468A46A342A5D130E7E9
:105FC000FB21E93F7BD9024000004054FB21F93F0F
:105FD0003163621A61B4D03DFB213941FFFFEF7F8D
:105FE000EAFBFFFF0000704188B3000083C8C96D61
:105FF000305FE43F0000E03F7370032E8A19A33B3B
:10600000C14920259A837B3908B30000D3220C4B69
:10601000520501F0C9FA0B4A0B4B04000D0001F0C8
:10602000C3FA02000B00414620000A604B602900C1
:1060300002F050F9034A044BB9E6032373E6C04665
:1060400061B4D03D7370032E8A19A33BF0B5474667
:10605000CE4680B587B000920193754B4F008146C4
:1060600088467F089F4263DC02F07CFC002800D158
:10607000D4E04A4643464846414601F0B9FE040092
:106080000D006C4A6C4B01F0B3FE6C4A6C4B01F096
:106090008BFA22002B0001F0ABFE6A4A6A4B02F039
:1060A00019F922002B0001F0A3FE684A684B01F0A9
:1060B0007BFA22002B0001F09BFE664A664B02F041
:1060C00009F922002B0001F093FE644A644B01F0B1
:1060D0006BFA22002B0001F08BFE0290039100224C
:1060E000604B2000290001F083FE029A039B06000A
:1060F0000F002000290001F07BFE009A019B0400A4
:106100000D004846414601F073FE02000B002000DE
:10611000290002F0DFF802000B003000390002F025
:10612000D9F802000B0000204F4902F0D3F870E0CC
:1061300002000B0001F05CFE04000D003D4A3E4BE6
:1061400001F056FE3D4A3E4B01F02EFA22002B0094
:1061500001F04EFE3B4A3C4B02F0BCF822002B0003
:1061600001F046FE394A3A4B01F01EFA22002B009C
:1061700001F03EFE374A384B02F0ACF822002B000B
:1061800001F036FE354A364B01F00EFA2B002200A4
:1061900001F02EFE354B029003919F429FDD344B60
:1061A00000229F423DDC334900207B182E49160017
:1061B0001F0002F08FF8049005910022294B200067
:1061C000290001F015FE32003B0002F083F8029A2C
:1061D000039B06000F002000290001F009FE009A31
:1061E000019B04000D004846414601F001FE0200FB
:1061F0000B002000290002F06DF802000B003000B7
:10620000390002F067F802000B000498059902F0CB
:1062100061F807B00CBC90469946F0BD00201249C9
:10622000F7E7154B002604920593144FC5E7C046C7
:10623000FFFF3F3ED43888BEE9FAA8BDC4B1B4BD63
:106240009EEE213EAD529C804F7E923E9015CB1922
:10625000A001FA3E7751C1166CC1563F4C555555B9
:106260005555A53F0000E03F0000F03F3233D33FDB
:106270000000E93F0000E0FF0000E73F0000D23FE0
:10628000F0B5DE464E4645465746E0B5DC4CA544E3
:106290000D9114001900A49A0993DA4B9200D65874
:1062A0004D1E03901821E01E0696029500F09EFEFA
:1062B000C3430100DB1719404B1C9A009B1ADB00FB
:1062C0001B190B9105934C1B771918D4A59BA5009E
:1062D0009C463F1922AE6544013707E0286802F06A
:1062E00077FB013403C60435BC4208D0002CF5DA34
:1062F00000200021013403C60435BC42F6D1069BC0
:10630000002B01DA00F0FDFB069B03990133DB0053
:106310009A46099BDA00944600920022914672AA9E
:106320000492B94A6144934688469AAB63449B44BD
:10633000029B002B00DABCE15D4600260027039C8F
:106340004D442A686B6803CC01F052FD02000B003B
:106350003000390001F028F9083D06000F004445DF
:10636000EFD1049B4B441E605F6008239C46E144D0
:10637000D145DDD10EA804218446494261448C46B2
:10638000069A93009C44614684460A910399083B0F
:1063900063448C460C93009B009263449B46009A96
:1063A0000498D10003008C46634408911E685F681E
:1063B000002A33DD954980468C466244D3009844D8
:1063C00070AB9A460EAB99460022914B30003900D3
:1063D00001F00EFD02F0C6FA02F0FAFA00228D4B2F
:1063E00004000D0001F004FD02000B003000390034
:1063F00001F070FF02F0B6FA4B4601C399464346DE
:1064000020001A685B68290001F0CEF808235B427F
:106410009C46E04406000F00D045D5D1059B3000D6
:106420001A003900984600F0DDFCFF2300229B058E
:1064300004000D0001F0DCFC00F038FC0022764B7B
:1064400001F0D6FC02000B002000290001F042FF01
:106450000D00040002F086FA814602F0B9FA02004B
:106460000B002000290001F035FF060040460F0018
:10647000002800DCEEE0009B18215A1E92000EABB3
:106480009B58091A1D000D41A9448D405D1B0EABA0
:106490009D5017231B1A1D41002D2DDD01239C4605
:1064A000009BE144002B00DC1CE20E9C0123002C2D
:1064B00000D0B5E0009A012A09D099000EAA5458DC
:1064C0000133002C00D0ACE0009A9A42F5D1059B34
:1064D000002B0EDD012B00D1A8E1022B09D1009B7E
:1064E0000EA95A1E92000EAB9B5807939B029B0A63
:1064F0008B50022D00D1C1E0002300223000390072
:1065000000F07EFE009B002800D194E2069A591EFE
:106510008A4210DC414A0A9894460EAA6344944683
:1065200000229B0063441C68043B22438342FAD14F
:10653000002A00D0C0E0069B0EAA013B9B00D35866
:10654000002B00D0B3E001220C9B043B59680132C0
:106550000029FAD0009B9C466244110007921A0061
:1065600001338B4246DC0B9863468046A59C43442E
:10657000A046099C9B00A1464A449844D30022AA05
:106580009146049A99449446089BA59A634484468C
:10659000614494469A468B0063440093434658688E
:1065A00002F016FA4B4618605960029B002B24DB60
:1065B0004D46039C0026002701E0286869680CCC42
:1065C00001F016FC02000B003000390000F0ECFF77
:1065D000083D06000F005C45EFD153469E60DF602A
:1065E00004239C460433E0449C46009BE144E2447F
:1065F0009845D3D1079B0093D1E600260027ECE70E
:1066000094FDFFFFD0B4000018FEFFFFFFFFFF1F47
:106610000000703E0000704100002040FFFFFF3F7F
:10662000002180225204141B0EAA54500099994252
:106630000EDD0EA884469B000EAA8900D258614444
:106640006344CF4800E01A68821A04C38B42FAD12F
:1066500001243CE7059B002B06D1009B0EAA013BC1
:106660009B00D558ED1517E70022C64B300000F00F
:10667000EBFD002800D024E100253DE732003B007F
:106680000020C14901F026FE06000F00002C00D1B9
:1066900032E7059A0020BC4900F0A4FB02000B0081
:1066A0003000390001F016FE06000F0024E7012239
:1066B00050E70026002754E64B46059A0793884684
:1066C0008B000EA9CB58183A08950592002B0DD1D6
:1066D0008C464146AD4B43449B006344043B5868A1
:1066E0000139183A0028F9D088460592059A002009
:1066F000A54900F077FB434604000D00002B00DAAB
:1067000005E29E000EAB9C464346DB0066449C4679
:10671000059370AB9946049F67440097306802F078
:1067200057F922002B0001F063FB002238607960EA
:10673000974B2000290001F05BFB083F04000D008F
:10674000043EB945EAD14AAB03939B4600239A46DF
:10675000069B4246994643460132029204934B46B9
:10676000002B00DAAAE080208A4B009D9846C005E5
:10677000894900260027002408E008239C460835A4
:10678000E044544511DC4346186859682A686B6830
:1067900001F02EFB02000B003000390000F004FF76
:1067A000013406000F00A145E7DA5B46C0C39B46F3
:1067B00001239C46009BE244083B0093029B9A45C0
:1067C000CDD1049B9846A49B022B00DD8EE0002BCC
:1067D00037DC1FD1059B00271D00039B00249C462E
:1067E0001E006544083E2A686B683800210000F0EE
:1067F000DBFE083D07000C00AE42F4D1089B002BE5
:1068000003D080231B069C4664443A0023000D9964
:106810000A604B600720079B18409B239B009D4408
:106820003CBC90469946A246AB46F0BD009B0EA9E3
:106830005A1E92000EAB9B5807935B025B0A8B506B
:1068400057E64346002B00DA70E100200021DB0010
:106850004AAAD61848AF32687368083E00F0A4FE12
:10686000B742F8D1089B002B00D025E10B000200B5
:106870004A984B990D9C2260636001F02BFD4346C2
:1068800007000C00002B13DD01254CAEB14638008B
:106890002E0021004C4601360CCC00F085FEA146AE
:1068A000B045F7DA089B07000C00002B00D015E17B
:1068B0003A0023000D998A60CB60ABE700260027E1
:1068C00073E701239C46009BE1440225002B00DD79
:1068D000EBE532003B0000202B4901F0FBFC0600F9
:1068E0000F0009E60024F2E54AAB0393A49B032BB7
:1068F00000D08FE74346002B00DC14E1039ADB0055
:106900009B46130091465B441E685F68234B4344DB
:106910000293DB00994448AB9A464B465C681B687F
:106920001800210032003B000090019100F03CFE75
:1069300004000D0002000B000098019901F0CAFC50
:106940003B00320000F030FE4B469860D9601C607E
:106950005D6008235B429C46E14426002F00CA4547
:10696000DBD14346012B00DCE3E0039A13005B44D8
:106970001E685F68029BDB0099464A44904610E01F
:10698000FFFFFF000000E03F0000F03FFFFFFF3F80
:106990000000703E90B40000FB21F93FFFFFFF1F95
:1069A000984643465C681B681800210032003B0093
:1069B0000090019100F0F8FD04000D0002000B00B2
:1069C0000098019901F086FC32003B0000F0ECFDDC
:1069D0004346039A9860D9601C605D60083B2600BE
:1069E0002F009A42DCD14D469446002600244746AB
:1069F000083565442A686B683000210000F0D4FD3A
:106A0000083D06000C00AF42F4D1039B4A9F5D682D
:106A10009968D868089B002B65D08022120694469E
:106A20000D9B6544604464441F605D609960D8605C
:106A30001E615C61EEE69A464B460793059B30006B
:106A40005A423900089500F0CDF900223A4B060071
:106A50000F0000F0F9FB002824D0384B0022300052
:106A6000390001F0C5F901F07DFF524604009500A0
:106A700001F0AEFF0022304B01F0BAF902000B002A
:106A80003000390001F026FC01F06CFF0EAA5051D5
:106A90000122059B524418339046059393000EAA99
:106AA000D45023E65346300039009C0001F05AFFD1
:106AB0000EAB1851D04619E680230D9A1B06CB1851
:106AC000106053600B0002004A984B9901F002FCE1
:106AD000434607000C00002B00DDD5E680231B0693
:106AE0009C466444E4E62B003A000D9D2A606B60EE
:106AF0000A000300AA60EB60320023002A616B6188
:106B000088E6099BDB00009372AB049332E4A49BFC
:106B1000022B00DDE8E6002B00DD92E600D079E6EE
:106B2000002700246AE6002600246EE700200021EA
:106B300098E60026340068E7000070410000703ECF
:106B4000F0B5CE46474680B587B000920193474ADC
:106B50004B00814688465B08934207DC4146484625
:106B600001F000FF4146031E484666D04A464346B0
:106B70004846414601F03CF904000D0002000B00BC
:106B80004846414601F034F9394A3A4B06000F00B5
:106B90002000290001F02CF9374A384B01F09AFB0C
:106BA00022002B0001F024F9354A364B00F0FCFCA2
:106BB00022002B0001F01CF9334A344B01F08AFB10
:106BC00022002B0001F014F9314B324A00F0ECFCAA
:106BD0000E9B02900391002B34D000980199002263
:106BE0002D4B01F005F9029A039B049005913000AA
:106BF000390001F0FDF802000B000498059901F03E
:106C000069FB22002B0001F0F3F8009A019B01F0D0
:106C100061FB224A04000D00214B3000390001F0D5
:106C2000E7F802000B002000290000F0BDFC020084
:106C30000B004846414601F04DFB07B00CBC9046A6
:106C40009946F0BD02000B002000290001F0D0F8A9
:106C5000124A134B01F03EFB32003B0001F0C8F832
:106C60004A46434600F0A0FCE7E7C046FFFF3F3E30
:106C70007CD5CF5A3AD9E53DEB9C2B8AE6E55A3EC6
:106C80007DFEB157E31DC73ED561C119A0012A3F62
:106C90001111813FA6F810110000E03F49555555EC
:106CA0005555C53F49004B0819007047474AF0B594
:106CB0004F4691464B005B0D99444646D6464A46A0
:106CC000C0B505000C000E0088460700132A27DC1B
:106CD000002A4BDB3E4B13419A460B0052461340B1
:106CE000034318D03B4A3C4B2800210000F05CFCD9
:106CF0000022002300F09EFA002847D0002C04DA7E
:106D000080234A465B031341984446465346002776
:106D10009E43380031001CBC90469946A246F0BD07
:106D2000332A08DD8023DB009945F4D102000B00F3
:106D300000F03AFCEFE7294A9446012263445242AC
:106D4000DA4092460242E6D0224A234B2800210034
:106D500000F02AFC0022002300F06CFA002815D075
:106D6000002C1EDB534646469F430FE0194A1A4B40
:106D70002800210000F018FC0022002300F05AFA3D
:106D8000002803D0002C04DB002700263800310047
:106D9000C1E76400640825430027002DF6D0104E9B
:106DA000F4E74B46142B0BD03422D21A0123934024
:106DB0005D19BD4208D201239C462F00E044D1E773
:106DC000133B9C46E044CDE72F00CBE701FCFFFFDF
:106DD000FFFF0F009C7500883CE4377EEDFBFFFF52
:106DE0000000F0BF4B0070B55B0D14000A00002BD3
:106DF0001AD14B005B08034315D0234B002200F04F
:106E0000F7FF224B9C422DDB0A004B005B0D363B0B
:106E10001F4DE318AB422ADC002B0DDD1D4C1B057A
:106E200022401A43110070BD1B4DAB42F0D102004D
:106E30000B0000F0B9FBF6E71D00353519DA174BEA
:106E400002009C4209DD0B001548164900F032F89B
:106E5000134A144B00F0CCFFE5E70B00124813492E
:106E600000F028F8104A114B00F0C2FFDBE70200E7
:106E7000E9E7084C363322401B0513431900002272
:106E80000B4B00F0B5FFCEE700005043B03CFFFFD6
:106E9000FE070000FFFF0F80FF07000050C3000047
:106EA0009C7500883CE4377E59F3F8C21F6EA5013B
:106EB0000000903C30B54A00DB0FDB0752081A4354
:106EC000110030BD02B4714649084900095C49000F
:106ED0008E4402BC7047C046002243088B4274D3E4
:106EE00003098B425FD3030A8B4244D3030B8B42CB
:106EF00028D3030C8B420DD3FF22090212BA030CD4
:106F00008B4202D31212090265D0030B8B4219D3B4
:106F100000E0090AC30B8B4201D3CB03C01A5241D4
:106F2000830B8B4201D38B03C01A5241430B8B421C
:106F300001D34B03C01A5241030B8B4201D30B0305
:106F4000C01A5241C30A8B4201D3CB02C01A52412C
:106F5000830A8B4201D38B02C01A5241430A8B42EF
:106F600001D34B02C01A5241030A8B4201D30B02D8
:106F7000C01A5241CDD2C3098B4201D3CB01C01AF2
:106F8000524183098B4201D38B01C01A52414309FC
:106F90008B4201D34B01C01A524103098B4201D3EA
:106FA0000B01C01A5241C3088B4201D3CB00C01A57
:106FB000524183088B4201D38B00C01A52414308CF
:106FC0008B4201D34B00C01A5241411A00D20146F4
:106FD000524110467047FFE701B5002000F0F0F87D
:106FE00002BDC0460029F7D076E7704703460B4341
:106FF0007FD4002243088B4274D303098B425FD3B2
:10700000030A8B4244D3030B8B4228D3030C8B42DD
:107010000DD3FF22090212BA030C8B4202D31212C3
:10702000090265D0030B8B4219D300E0090AC30B98
:107030008B4201D3CB03C01A5241830B8B4201D345
:107040008B03C01A5241430B8B4201D34B03C01A2E
:107050005241030B8B4201D30B03C01A5241C30AA6
:107060008B4201D3CB02C01A5241830A8B4201D317
:107070008B02C01A5241430A8B4201D34B02C01A01
:107080005241030A8B4201D30B02C01A5241CDD2A6
:10709000C3098B4201D3CB01C01A524183098B42F1
:1070A00001D38B01C01A524143098B4201D34B01DA
:1070B000C01A524103098B4201D30B01C01A52413D
:1070C000C3088B4201D3CB00C01A524183088B42C4
:1070D00001D38B00C01A524143088B4201D34B00AD
:1070E000C01A5241411A00D201465241104670471F
:1070F0005DE0CA0F00D04942031000D34042534024
:1071000000229C4603098B422DD3030A8B4212D3E3
:10711000FC22890112BA030A8B420CD38901921115
:107120008B4208D3890192118B4204D389013AD052
:10713000921100E08909C3098B4201D3CB01C01A27
:10714000524183098B4201D38B01C01A524143093A
:107150008B4201D34B01C01A524103098B4201D328
:107160000B01C01A5241C3088B4201D3CB00C01A95
:10717000524183088B4201D38B00C01A5241D9D2AD
:1071800043088B4201D34B00C01A5241411A00D22E
:107190000146634652415B10104601D34042002B2A
:1071A00000D54942704763465B1000D3404201B5A9
:1071B000002000F005F802BD0029F8D016E770475E
:1071C0007047C046D0400B1C1141203A03D49C4666
:1071D0001341184363465242934018437047C046D8
:1071E0008446101C62468C46191C634600E0C0466B
:1071F0001FB500F095FD002801D40021C8421FBD35
:1072000010B500F0EDFC4042013010BD10B500F0AB
:1072100087FD002801DB002010BD012010BDC04605
:1072200010B500F07DFD002801DD002010BD01201B
:1072300010BDC04610B500F00FFD002801DC002095
:1072400010BD012010BDC04610B500F005FD00289E
:1072500001DA002010BD012010BDC046F0B5CE46B9
:10726000474615042D0C2E0080B50704140C3F0C66
:107270009946030C7E435D43674363437F19340C97
:10728000E4199C46A54203D980235B029846C44476
:107290004B4643435143250C36046544360C2404C5
:1072A000A4195B19591820000CBC90469946F0BDF2
:1072B000F0B54E4657464546DE46E0B543025B0A0A
:1072C000450083B00F1C99462D0EC60F002D57D0D8
:1072D000FF2D24D08020DB00C0041843002381460A
:1072E0009A469B467F3D7C027A00FB0F640A120E91
:1072F000984623D0FF2A4BD0E30080240020E404EA
:107300007F3A1C43AD186B1C4746019353467740A8
:107310003A000F2B48D87D499B00CB589F46002B45
:1073200000D085E008339A46063B9B467C027A00F3
:10733000FB0FFF25640A120E9846DBD1002C00D00B
:1073400090E0524601231A4392460120DBE74C4667
:1073500058461700022824D0032800D1CFE000228D
:10736000002301284DD15802D205400AFF071043DF
:10737000384303B03CBC90469946A246AB46F0BDAC
:10738000002B5BD104239A46033B00259B46AAE7CA
:10739000FF35002C60D1524602231A439246022048
:1073A000B1E7FF220023DEE74B461B0C9C464B4611
:1073B0002604360C180461463300220C6446000C87
:1073C00043434E435043544380191A0C12189642BB
:1073D00003D9802149028C4664441B041B0C100411
:1073E000C01883015E1EB341800E1843130C1B1995
:1073F0009B0103431C00230179D5012362081C4033
:107400001443019A7F32002A4DDD630704D00F2315
:107410002340042B00D00434230103D53C4B019AB4
:107420001C408032FE2ABCDCA3015B0AD2B29AE780
:107430000C239A46093BFF259B4654E7180001F0B0
:1074400053FB4A46431F76259A4000236D429146DE
:107450002D1A9A469B4646E7524603231A43924604
:10746000032050E7200001F03FFB431F2D1A9C40F2
:10747000763D002047E780230027DB03FF2272E7E9
:10748000424666E74C463200584662E780234A4649
:10749000DB031A4222D01C4220D123435B025B0A49
:1074A0004746FF225FE701239A1A1B2A21DC2300AB
:1074B0000199D3409E318C401A0023005C1EA341E9
:1074C00013435A0704D00F221A40042A00D0043371
:1074D0005A0111D49B015B0A002244E780234A46EB
:1074E000DB0313435B025B0A3700FF223BE7019596
:1074F00087E70022002336E70122002333E78023B9
:10750000DB0323435B025B0AFF222CE7E0B40000AD
:10751000FFFFFFF770B500283DD0C317C5185D40C9
:10752000C40F280001F0E0FA9E22121A962A07DC06
:10753000D2B2082833DD083885406802400A23E0CB
:10754000992A0BDD052329001B1AD94003001B33A0
:107550009D402B005D1EAB4119430D00052801DD48
:10756000431F9D402B000F490B406E0709D00F268B
:107570003540042D05D004335D0102D59F220B4018
:10758000121A9B01580AD2B24002D205400AE407FF
:107590001043204370BD002400220020F4E768025D
:1075A000400AF1E7FFFFFFFBF0B54F464646D646DF
:1075B0000C000903C0B5490A470F5E0039431F0399
:1075C000DB0F9C4665007B0A570F1F436D0DE40FD0
:1075D000760DA146C000B846D200AB1B64457BD0F7
:1075E000002B5FDD002E00D0A4E03E00164300D14A
:1075F00012E15E1E002E00D09EE1871A4346B8427B
:1076000080410125C91A4042091A0B0200D431E118
:1076100049024E0A002E00D16EE1300001F064FAFA
:107620000300083B1F2B00DD61E120223900D21A44
:107630009E40D1409F400E439D4200DD51E15D1BC5
:107640006B1C1F2B00DD7CE12021C91A3D0030009E
:107650008F408840DD40791E8F413100072228434A
:10766000D940002507433A40002A09D00F233B4068
:10767000042B05D03B1DBB42BF417F42C9191F00EF
:107680000B0200D426E26A1CC64B55056D0D9A42CA
:1076900000D106E1C44AFF080A40530752023B43A7
:1076A000120B8EE0002B00D0B8E06B1C5B055B0D6D
:1076B000012B00DC30E1871A4346B842B641CB1AB1
:1076C00076429E1B330200D54CE13B003343A1D1EF
:1076D00000220024002570E0002B00DCE5E0002EF5
:1076E00000D183E0AF4EB54260D0802636043743E8
:1076F000B846382B00DC3EE1434613431F007A1E98
:1077000097413F1887428041404209180B0200D43C
:10771000B0E0A44B01359D4200D1C3E0A24A7B08F2
:107720000A4001210F401F435108D30707221F437E
:107730003A4099E79B4EB54238D08026360437430D
:10774000B846382B00DDDCE01F2B00DC30E11E00EA
:107750004746203EF740BC46202B04D04026F31A73
:1077600046469E403243170063467A1E97411F43A8
:10777000CCE0002B00D104E24346134300D159E191
:107780004B07C00818438023C9081B03194208D0BF
:107790004546ED081D4204D14346D0085907084329
:1077A0002900420FC9007F4D1143C0004B07CA0892
:1077B0007C49C00803438D4268D012036D05120B4B
:1077C0006D0D002112031800130B0A0D12051A4348
:1077D000764B2D0513402B435B00E4075B082343E6
:1077E00019001CBC90469946A246F0BD3E001643C7
:1077F00012D05E1E002E00D000E187188742804123
:1078000041444042091801250B0233D5022585E782
:1078100064463300414610001D00C7E7002D00D02C
:10782000DAE00C000443F3D05C1C00D19FE15D4C16
:10783000A64200D12FE1DB43382B00DD66E11F2B90
:1078400000DD83E120240500E41A0F00DD40D9406B
:10785000A0404346A7405B1A441EA04198462F43D0
:107860003843171ABA42924143465242991A644623
:107870003500CAE607223A40002A00D0F6E64B0758
:10788000CA084849FF083B438D4296D1190011436D
:1078900000D19EE1802109030A431203120B414DDE
:1078A0008FE71500002200238BE7002B00D0C7E0F4
:1078B0006B1C5F057F0D012F00DCF1E0394DAB4201
:1078C00000D1B9E085180A00854289414244494205
:1078D00051180722CF076D082F4349083A401D0071
:1078E000C2E607223049ED1A31403A40BCE63E007C
:1078F0002838864000279FE6380001F0F5F8203050
:107900008EE6434613431F007A1E9741C71BB842B9
:1079100080414042091A78E60E003B0006431343BB
:10792000002D61D1002E00D0F4E0002B00D11BE12E
:1079300064463900100039E71A4FBB427AD0330051
:10794000FFE630001F3DE840202B03D04021CB1A3A
:107950009E4037437B1E9F41072207433A40002148
:10796000002589E7171A4346BA42B641591A7642AA
:107970008E1B64464EE61F2B00DDADE020264746F9
:10798000F61AB740B9461700B246DF404E463E43AE
:1079900037005646B240561EB24117434246DA40BF
:1079A0008918AEE6FF070000FFFF7FFFFFFF0F8093
:1079B00020264746F61AB740B9461700B246DF40C0
:1079C0004E463E4337005646B240561EB24117431C
:1079D0004246DA40891A99E77F4CA6425BD0802460
:1079E00024045B42214327E7002E0CD1002B00D159
:1079F000CBE0644639001000774DD7E6764FBB42A6
:107A000018D0330075E6002B14D04B07C00818437C
:107A10008023C9081B03194207D0FC081C4204D16B
:107A20007907D0080843E14621004C46420FC900BF
:107A30001143C000684DB9E61D0000220023C0E6D6
:107A4000002D5BD10D00054300D1E2E65D1C00D1A5
:107A5000B0E0614DAE421FD0DB43382B71DC1F2BF1
:107A600000DD96E020250F00ED1AAF40B946070073
:107A7000AA46DF404D463D432F005546A840D94019
:107A8000451EA84188440743BF189742924151427E
:107A9000414435003AE6644635004146100085E62B
:107AA0000B000343002D00D063E6002BF5D04346C6
:107AB000134300D17AE68718874280410722414468
:107AC000404209183A400B0200D4D5E6434B013539
:107AD0001940C9E5380069E61E004746203EF740D8
:107AE000BC46202B04D04026F31A46469E40324323
:107AF000170063467A1E97411F4302E6364DAE4299
:107B0000CAD080252D045B422943A6E70843411EC5
:107B10008841A6E6002B00D148E6871A4346B842C2
:107B2000B641CB1A76429E1B33024BD5171A4346F9
:107B3000BA429241591A5242891A072264463A407F
:107B400092E501430F00791E8F419DE71C000F0055
:107B5000203CE740202B03D04024E31A99400843FF
:107B6000411E884138437CE60022002425E6171A8E
:107B70004346BA429241591A5242891A6446350024
:107B800043E541461000144D10E680220024120304
:107B900080E61D000F00203DEF40BC46202B03D0A7
:107BA0004025EB1A9940084307006346781E874139
:107BB0001F4369E7871897429B4141445B42C918BC
:107BC0003500A3E53B003343CED0072231003A40D5
:107BD00052E600231A00F4E5FF070000FFFF7FFFD5
:107BE000F0B54F464646D6468446C0B58046194E47
:107BF00018030F034D00000B5C0082463F0B6D0D18
:107C0000C90F9146640DDB0F0120B5420AD0B44282
:107C100003D0A54201D157450CD01CBC90469946D3
:107C2000A246F0BD66463E43F7D1AC42F5D154467C
:107C30001443F2D10120C845EFD1994207D0002D5D
:107C4000EBD163461F433800471EB841E5E70020EB
:107C5000E3E7C046FF070000F0B54F464646D6466C
:107C60004D00C0B50E03C90F8A462C491F035C00A6
:107C70008046360B6D0D91463F0B640DDB0F8D4238
:107C80001ED08C4216D0002D1ED130438446002CCD
:107C900001D13A4323D06246002A1AD09A4529D00E
:107CA000514602200139084001381CBC90469946D3
:107CB000A246F0BD39001143E5D002204042F4E76E
:107CC0003043FAD1AC420FD0002C0FD13A43E7D069
:107CD0000CE00122013B934318000130E5E76346C5
:107CE0000020002BE1D0DBE73A43E6D19A45D7D11B
:107CF000A542D5DCA54205DBBE42D1D808D0002084
:107D0000BE42D2D250460123013898430130CCE71D
:107D1000C845C5D80020C845F4D3C6E7FF07000012
:107D2000F0B54F464646D6464D00C0B50E03C90FC6
:107D30008A462E491F035C008046360B6D0D914626
:107D40003F0B640DDB0F8D4218D08C4211D0002DFB
:107D500018D130438446002C1ED13A431CD16346CF
:107D60000020002B30D05146022001390840013854
:107D70002AE039001143EAD0022025E03043FBD14C
:107D8000AC4226D0002C26D13A4324D151460220C1
:107D900001390840013817E06246002A0FD09A45A1
:107DA000E1D1A54205DBBE42DDD819D00020BE429C
:107DB0000AD25046012301389843013004E00122E1
:107DC000013B9343180001301CBC90469946A246E3
:107DD000F0BD3A43D0D19A45C5D1A542C3DCE0E716
:107DE000C845C0D80020C845E3D3EDE7FF07000031
:107DF000F0B55746DE464E464546E0B5834606009A
:107E00000F03480087B092461D003F0B400DCC0F7A
:107E1000002800D16FE0DE4B984238D08023FF006D
:107E20001B041F43730F3B430193DA4B0027994612
:107E300000239B46F60081442B0369001B0B52462E
:107E40009846490DED0F002900D185E0D04B9942AD
:107E500000D173E04346DA0080231B0413435246EB
:107E6000CC48520F84461343524600206144D2004E
:107E700089442100694000918C46012149448A4689
:107E80000F2F00D990E0C449BF00CF59BF465B46D1
:107E90003B43019300D06AE1022308270026814674
:107EA0009B46C9E732005846019B61460091022873
:107EB00000D175E0032800D1FEE1012800D02CE1BB
:107EC00000230027002600253F032A0D3F0BB3485F
:107ED00012053A4302401B051343009A5B00D10789
:107EE0005B080B433000190007B03CBC9046994634
:107EF000A246AB46F0BD5B463B43019300D12FE168
:107F0000002F00D1A5E1380000F0EEFD03000B3B8F
:107F10001C2B00DD96E11D22D31A5A460100DA40DF
:107F20005E4608398F4013008E403B4301939C4BC3
:107F300000271B1A994600239B467DE7414653467E
:107F40000B4393498C46E144002B00D01AE10222F6
:107F50000220174300228CE7134300D10DE1434672
:107F6000002B00D181E1404600F0BEFD02000B3A3B
:107F70001C2A00DD72E10100434608398B40984617
:107F80001D239A1A5346D3401A00434613435246C0
:107F90008A404946081A824989468144002068E798
:107FA0007B4B002700268EE7140C1204120C1100E4
:107FB000370C3604350C794328008C462E0060437C
:107FC0006044834656432100300C8046584679432E
:107FD00040440291844506D98846802149028C4656
:107FE000E044414602913604010C360C00048B46F5
:107FF00081191E0C1B041B0C0391190079438C463C
:10800000280075436544A8465843050C454477430A
:10801000A94203D9802149028C466744290C8C4629
:1080200039000004000C2D042D186144AB44059167
:108030005946049101990F043F0C080C3900514333
:108040004243904602008C46090C8B4662437C43B7
:1080500044445C44A04503D98021490288464244F7
:10806000210C884661460904090C8C4639005943A5
:10807000434370437E430F0CF6182404BE19644436
:1080800042448C46B34203D980235B029846404465
:10809000029B61469846049B370443449B46AB458C
:1080A000AD416B420D0405992D0C8C467F19674438
:1080B000FD18A8465D462D19A542A4419346644289
:1080C000A446C344DC448F42BF4198459B4193453D
:1080D0009241A445A4415B427F421F43360C524269
:1080E0006442BF192243BF18624638184302D20DBA
:1080F000039913436A020A43501E82416146ED0D03
:108100002A434E023243D90100D4B3E0012650087D
:1081100032400243DE0732435B08224C5444002CB9
:1081200062DD510709D00F201040042805D0101D32
:108130009042924152429B180200D90104D58024FA
:108140001948E400034054441848844200DD27E7FE
:108150005E075B02D2081F0B630516435B0DB2E698
:10816000002399460133042700269B4664E6032337
:10817000019781460C279B465EE6012201201743AA
:10818000002276E6032303201F43434671E6C046E0
:10819000FF07000001FCFFFF20B50000FFFF0F807C
:1081A0000DFCFFFFFF030000FFFFFFFEFE070000C6
:1081B0000023802700933F030026434B83E6019B67
:1081C0003200A446584670E6AC466EE68027019918
:1081D0003F0339422DD03B422BD11F433F033F0B7E
:1081E00000951600384B6EE601252D1B382D00DD5D
:1081F00066E61F2D40DC35481C00504416008240C6
:108200008440EE40501E824134431443EB406207E9
:1082100009D00F222240042A05D02200141D9442C6
:10822000804140421B181A023ED501230027002638
:1082300049E68027019B3F031F433F033F0B009408
:10824000214B40E603005A46283B9A400026019203
:108250006DE6584600F048FC203057E603005246D1
:10826000283B9A401300002293E6504600F03CFC65
:1082700020307BE6CA4650E71F201E004042041B08
:10828000E640202D03D0124C5444A3401A43501E04
:108290008241324307260027164009D00F200023D1
:1082A000104014000428B9D122005E075B021F0BA6
:1082B000D2081643002306E680273F031F433F03EF
:1082C0003F0B1600004BFEE5FF0700001E040000F8
:1082D0003E040000F8B557464E464546DE460C00C3
:1082E0000903E0B5490A460F5F0031431E03DB0F67
:1082F000760A9B46530F3343C84E6500C000E40F17
:10830000D2006D0DA24681467F0D9C469046B74235
:1083100000D1B9E05B46012673409B46EE1BA345A6
:1083200000D183E0002E63DD002F00D0B1E0634672
:10833000134300D123E1731E002B00D0BAE1861A4B
:108340006346B04280410125C91A4042091A0B0216
:1083500000D447E149024B0A98464346002B00D11E
:1083600089E1404600F0C0FB0300083B1F2B00DD05
:108370007CE120223000D21A4146D04099400200D0
:108380009E400A439D4200DD6AE15D1B6B1C1F2B72
:1083900000DD94E1202110003500C91A8E40DA403A
:1083A0008840DD40711E8E411100072228430025C0
:1083B00006433240002A09D00F233340042B05D056
:1083C000331DB342B641764289191E000B0200D418
:1083D0003DE26A1C914B55056D0D9A4200D119E1A1
:1083E0008F4AF6080A40570752023743120B9BE0A8
:1083F000002E00D0C5E06E1C7605760D012E00DC47
:1084000048E16746861ACB1BB042BF417F42B8465F
:108410001F004346FF1A3B00B8461B0200D55FE130
:1084200037439AD100220024002579E0002E00DC99
:10843000FAE0002F00D18DE0784B9D4267D0802379
:1084400067461B041F43BC46382E00DC52E16346DE
:1084500013435A1E93411E18864280414042091818
:108460000B0200D4BEE06D4B01359D4200D1D2E03D
:108470006B4A73080A4001210E401E435108D3077E
:1084800007221E43324095E71E00164300D045E701
:1084900040E7624B9D423AD0802367461B041F434E
:1084A000BC46382E00DDEBE01F2E00DC3AE1330045
:1084B0006746203BDF403B00202E05D04027BF1BF6
:1084C0006646BE40324390464646721E964133434E
:1084D000DAE0002B00D114E26346134300D168E1D7
:1084E00080234E07C008C9081B030643194208D061
:1084F0006046C008184204D163460100D2085E07F6
:108500001643F3009946C900720F444D11434B4680
:10851000DE08424B4F073743CA089D4200D16EE048
:1085200012036D05120B6D0D00211203130B0A0DC2
:1085300012051A433B4B2D0513402B435B00E40708
:108540005B082343380019003CBC90469946A2467C
:10855000AB46F8BD6346134311D0731E002B00D009
:1085600007E186188642804161444042091801258E
:108570000B0237D502257BE73E0061469146350068
:10858000C5E75C46002D00D0E1E00B000343F3D0CB
:10859000731C00D1ACE1214B9F4200D13AE1F3437F
:1085A000382B00DD6FE11F2B00DD8CE120250E0054
:1085B000ED1AAE40B0460600AA46DE4045463543B9
:1085C0002E005546D940A8406346451EA8415B1A77
:1085D0009C463043161AB242924163465242991A5F
:1085E0003D00B4E607223240002A00D0E4E60B4BFF
:1085F000F6084F073743CA089D4200D090E73B007A
:10860000134300D1A6E180231B031A431203120B6C
:10861000024D89E715000022002785E7FF070000CB
:10862000FFFF7FFFFFFF0F80002E00D0C7E06B1C15
:108630005E05760D012E00DCF0E0C84DAB4200D1A6
:10864000B9E085180A0085428941624449425118BF
:108650000722CE076D082E43490832401D00A9E6C7
:10866000BF49ED1A114007223240A3E632002838F4
:108670008240002686E6300000F036FA203073E6AD
:10868000634613435A1E9341C61AB042804140428A
:10869000091A5CE60E00674606431743002D5ED1BB
:1086A000002E00D0F3E0002F00D11EE15C466146B1
:1086B00091462CE7A94FBE427BD01E00F1E6100088
:1086C0001F3DE840202B03D04021CB1A9A4016438F
:1086D000731E9E410722064332400021002583E796
:1086E000161A6346B2428041591A40420B1A984604
:1086F0005C4632E61F2E00DDABE02027BB1B9A460E
:1087000063465746BB40994613004F46F3401F430C
:108710003B005746BA40571EBA4113436246F240E7
:10872000891898E62027BB1B9A4663465746BB40EC
:10873000994613004F46F3401F433B005746BA404B
:10874000571EBA4113436246F240891A9CE7834B95
:108750009F425FD080252D047342294320E7002EDD
:108760000CD1002F00D1D0E05C46614691467B4D94
:10877000CDE67A4FBE421CD01E0065E6002F18D011
:10878000C0084E0706438020C9080003014208D0F4
:108790006346DC08044204D12100DA46D2085E07B1
:1087A0001643F300994601245346C900720F114342
:1087B0001C406A4DABE61D0000220027B4E6002DE8
:1087C00059D10B00034300D1D6E6731C00D1B2E0AF
:1087D000624B9F421ED0F343382B6FDC1F2B00DD12
:1087E00097E020250E00ED1AAE40B0460600AA46DE
:1087F000DE40454635432E005546A840D940451E2B
:10880000A8418C440643B6189642924151426144B5
:108810003D0025E63D006146914678E60B000343A6
:10882000002D00D055E6002BF5D06346134300D150
:108830006DE6861886428041614440420918002254
:108840000B0200D4D0E6464B01351940B2E5B146E3
:108850005DE633006746203BDF403B00202E05D01D
:108860004027BF1B6646BE40324390464646721EB6
:1088700096413343EFE5394B9F42CBD080252D0401
:1088800073422943A8E70843411E8841A2E6002F0E
:1088900000D13CE66346861ACF1AB0429B415B4248
:1088A000FB1A98461B024ED5161A6346B2429241F5
:1088B000591A5242891A5C4600227BE501430E0098
:1088C000711E8E419FE71D000E00203DEE40B04618
:1088D000202B04D04025EB1A994008438146484696
:1088E0004346411E8841184374E60022002417E6DF
:1088F000161A6346B2429241591A5242891A3D00F1
:1089000025E561469146154D01E6802200241203BB
:1089100079E61D000E00203DEE40B046202B04D02D
:108920004025EB1A9940084381464E464346711E46
:108930008E411E4367E7861896429B4161445B4225
:10894000C9183D008CE547463743CED00722414643
:10895000324049E600273A00E6E5C046FF0700003E
:10896000FFFF7FFF30B5144D0A034B00120B5B0D68
:10897000C90F0024AB4211DD104CA34210DC80244F
:10898000640322430E4CE41A1F2C0CDD0D48C31A5D
:10899000DA4013005C42002900D11C00200030BDE9
:1089A000094BCC18FAE7094DE040AC4663449A40C5
:1089B00013000343EEE7C046FE0300001D04000061
:1089C0003304000013040000FFFFFF7FEDFBFFFFF7
:1089D00070B500282DD0C317C5185D40C40F2800FE
:1089E00000F082F8154B1B1A5B055B0D0A2815DD9C
:1089F0000B38854000222D032D0B002110002D0384
:108A00000A0D2D0B12052A430D4D1B052A40134359
:108A10005B00E4075B082343190070BD02002900D6
:108A2000153291400A000B21081AC5402D032D0B69
:108A3000E3E70024002300250022DEE71E040000F7
:108A4000FFFF0F804100090E4B1C70B5DBB24602E0
:108A5000750AC40F012B14DDE0239B006D07360B54
:108A6000CB1800210A0D280012051C4D32435B056E
:108A70002A405B0813435B00E4075B0823431900AB
:108A800070BD002914D1002D1ED0280000F02CF854
:108A90000A281CDC0B232A001B1ADA4003001533BA
:108AA0009D400F4B12031B1A5B05160B5B0DD8E79D
:108AB000002D06D0320B802636036D071643094B76
:108AC000CFE7084B0026CCE700230026C9E70300C8
:108AD0002A000B3B9A400025E3E7C046FFFF0F80CA
:108AE00089030000FF0700001C2101231B0498429A
:108AF00001D3000C10391B0A984201D3000A08392F
:108B00001B09984201D30009043902A2105C4018E5
:108B10007047C04604030202010101010000000089
:108B20000000000030B51C00094B05001B6885B033
:108B3000D868084B002A01D1074B1A000292019312
:108B400000912B002200054900F020F800F0FAFD0A
:108B50006400002060B50000BFA400006DB50000F7
:108B6000084B10B50400002B02D0002100E000BF2C
:108B7000054B1868836A002B00D09847200001F04D
:108B800005FBC046000000009CB500000EB403B514
:108B9000010003AB044804CB0068019300F020F906
:108BA00002B008BC03B018476400002070B500266E
:108BB0000C4D0D4C641BA410A64209D1002601F0F7
:108BC000E7FA0A4D0A4C641BA410A64205D170BDF9
:108BD000B300EB5898470136EEE7B300EB589847DF
:108BE0000136F2E734020020340200203402002073
:108BF0004402002010B5034B0100186800F06AF829
:108C000010BDC0466400002010B5034B0100186879
:108C100000F016F810BDC04664000020002310B517
:108C20009A4200D110BDCC5CC4540133F8E7030074
:108C30001218934200D1704719700133F9E7000010
:108C400070B50500002910D00C1F2368002B00DA36
:108C5000E418280000F0A8FF1D4A1368002B05D176
:108C600063601460280000F0A0FF70BDA34209D922
:108C7000216860188342F3D118685B68411821604D
:108C8000EEE713005A68002A01D0A242F9D9196808
:108C90005818A0420BD12068091858181960824250
:108CA000E0D110685268411819605A60DAE7A042B2
:108CB00002D90C232B60D5E721686018824203D1CA
:108CC000106852684118216062605C60CAE7C04663
:108CD0000C120020032370B5CD1C9D4308350600FF
:108CE0000C2D1ED20C25A9421DD8300000F05CFFCF
:108CF000254A14682100002919D1244C2368002B2F
:108D000003D1300000F02AFB20602900300000F081
:108D100025FB431C2BD10C233000336000F045FFB2
:108D200003E0002DDFDA0C233360002070BD0B68F8
:108D30005B1B19D40B2B03D90B60CC18256003E007
:108D40004B688C420DD11360300000F02EFF2000E4
:108D500007220B30231D9043C31AE7D05A42E2503A
:108D6000E4E763600C00EFE70C004968C3E7032306
:108D7000C41C9C43A042E1D0211A300000F0EEFA5E
:108D8000431CDBD1C7E7C0460C12002010120020A4
:108D9000936810B5013B9360002B04DA9469A342F9
:108DA00007DB0A2905D01368581C106019700800E9
:108DB00010BD00F0FBFB0100F9E7F8B506000F005D
:108DC0001400D518AC4201D1002007E021783A0008
:108DD0003000FFF7DDFF0134431CF3D1F8BD000084
:108DE000F0B59FB002900F0016000593002805D043
:108DF00083690493002B01D100F0A4FD7B4B9F42BB
:108E00005BD1029B5F68BB891B0762D53B69002B66
:108E10005FD0002306AC6361203363761033A37602
:108E200035002B78002B01D0252B5CD1AB1B049394
:108E30000CD0320039000298FFF7BFFF431C00D16D
:108E4000C4E06269049B9446634463612B78002B01
:108E500000D1BBE0012200235242626002A95432D9
:108E600052186E1C2360E360A3601370A365317811
:108E700005225F4800F07AFE751C002835D1226873
:108E8000D30604D5532302A95B18202119701307B8
:108E900004D5532302A95B182B21197033782A2B90
:108EA0002CD0350000210A20E3682A786E1C303A65
:108EB000092A64D900292ED026E04E4B9F4202D1C8
:108EC000029B9F689FE74C4B9F429CD1029BDF68AF
:108ED00099E73900029800F0BFFB002899D00120E3
:108EE00040421FB0F0BD01359BE7414B2268C01ADC
:108EF00001238340134323602E00B8E7059B191D0F
:108F00001B680591002B01DB099304E05B42E360E1
:108F10000223134323602B782E2B0AD16B782A2B44
:108F200035D1059B02351A1D1B680592002B2BDBE2
:108F30000793324E29780322300000F017FE0028F4
:108F400006D04023801B83402268013513432360F1
:108F5000297806222A486E1C217600F007FE002898
:108F60003AD0284B002B25D10722059B073393438A
:108F7000083305936369039A9B18636150E7434381
:108F800001219B18350090E701235B42D0E70023C5
:108F90000A201A000135636029786E1C30390929CE
:108FA00003D9002BC5D00792C3E7424301235218CF
:108FB0003500F1E705AB00933A00134B210002980E
:108FC00000E000BF0390039B0133D3D1BB895B0654
:108FD00000D584E70B9884E705AB00933A000A4B71
:108FE0002100029800F080F8ECE7C046F4B50000DC
:108FF000A0B5000014B60000D4B50000A6B500006E
:10900000AAB5000000000000BB8D0000F7B51500F8
:1090100001938A680B6900900C00934200DA1300F8
:1090200022002B6043321278002A01D001332B60DA
:1090300023689B0602D52B6802332B600627236822
:109040001F4027D0230043331B785A1E93412268C8
:10905000920630D42200019943320098089EB0470E
:10906000431C25D0062320682A68E16803400025B8
:10907000042B03D18D1AEB43DB171D40A368226933
:10908000934201DD9B1AED180027BD4220D100203C
:1090900010E00137E3682A689B1ABB42D2DD220048
:1090A0000123193201990098089EB047431CF0D162
:1090B00001204042FEBD3020E118433108702100FC
:1090C0005A1C45310978A218433202331170C1E7A6
:1090D000220001231A3201990098089EB047431CD0
:1090E000E6D00137D1E70000F0B589B004920A005C
:1090F00043320593039002920A7E0C000E9B6E2A67
:1091000000D186E01FD8632A33D008D8002A00D1C6
:109110008CE0582A4DD0250042352A7030E0642A70
:1091200001D0692AF7D1196825680A1D280629D5B2
:1091300008681A60002803DA2D23029A404213704F
:109140006B4E0A274FE0732A74D008D86F2A1FD0BD
:10915000702AE0D1202209680A43226003E0752AC0
:1091600016D0782AD7D12200782145321170614E6D
:1091700022E025001A684235111D196013682B7012
:10918000012365E008681A606906D3D500B2D1E70B
:1091900019682568081D186008682E0605D5544E04
:1091A00008276F2A1BD00A2719E06D06F7D580B271
:1091B000F5E745314E4E0A7018682268011D0068B7
:1091C0001960150621D5D30702D520231A43226042
:1091D0001027002803D1202322689A43226023000D
:1091E000002243331A706368A360002B58DB04220B
:1091F000216891432160002854D1029D002B5AD050
:109200002500337842352B7055E05506DBD580B20A
:10921000D9E71A680D68101D4969186013682E0691
:1092200001D5196002E06D06FBD519800023029D6F
:1092300023614FE01A68111D1960156800216268EA
:10924000280000F093FC002801D0401B6060636898
:1092500023610023029A13703CE023692A000499D9
:109260000398059DA847431C3ED023689B0715D44F
:10927000079BE068984239DA180037E022000123A2
:10928000193204990398059EB047431C2CD0013530
:10929000E368079A9B1AAB42F0DCE9E70025F7E7A1
:1092A0000028ADD0029D3900FDF79CFE735C013DA6
:1092B0002B700028F7D1082F09D12368DB0706D5CA
:1092C00063682269934202DC3023013D2B70029BCC
:1092D0005B1B2361059B07AA00932100049B039855
:1092E000FFF794FE431CB8D10120404209B0F0BD05
:1092F000B1B50000C2B50000124B10B51C68A36BDD
:10930000002B0FD11820FFF775FC0F4BA0630360F3
:109310000E4B012243600E4B83600B23838100239D
:1093200002614361A46B0B4A206961690A4BFDF736
:1093300095FF012200238018594120616161480096
:10934000400810BD640000200E33CDAB34126DE632
:10935000ECDE05002D7F954C2DF45158002370B59F
:10936000064C05000800236000F0FAFE431C03D100
:109370002368002B00D02B6070BDC046C4250020A0
:109380000CB430B5164B9DB00C1E1D6808DA8B234B
:1093900001202B6040421DB030BC08BC02B0184711
:1093A000822302A99B008B810023029008619C42CA
:1093B00000D0631E8B604B6101235B42CB81209AFE
:1093C00021AB2800019300F079FC431C01DA8B23C8
:1093D0002B60002CDFD00023029A1370DBE7C0461D
:1093E000640000200EB400B50B499CB01DAB029088
:1093F0000690079104910948094904CB059100683A
:1094000002A9019300F05AFC0023029A13701CB0C9
:1094100008BC03B01847C046FFFFFF7F6400002070
:109420000802FFFF02780B78002A03D001300131D7
:109430009A42F7D0D01A704703000A7801311A70A7
:109440000133002AF9D170470023C25C0133002A9E
:10945000FBD1581E704730B50500002A00D130BD41
:109460000C78013A6B1C2C700131002C05D19A1834
:109470009A42F4D01C700133FAE71D00EDE70000BA
:10948000F0B51F000E0087B00590019102920C9874
:10949000347800F0EAFA082200194378751C13406A
:1094A00036D12D2C36D1B51C74780126002F62D010
:1094B000102F09D1302C07D120222B789343582B21
:1094C00054D110276C7802352D4B3900F318180051
:1094D0000393FDF787FD0491012100234942020017
:1094E0008C4618002100303909291AD80C00A742EF
:1094F00023DD591C09D06346824206D302D1049968
:10950000A14202DB0123784320182C780135E9E7DA
:109510002E00BCE72B2C01D01E00C7E7B51C7478C9
:10952000FAE721004139192901D8373CDFE721004A
:109530006139192901D8573CD9E75A1C08D1059A35
:1095400023331360029B0398002B09D107B0F0BDB1
:10955000002E00D04042029A002AF7D0002B01D002
:109560006B1E0193029B019A1A60EFE73024002FD3
:10957000AAD10827A8E7302C9ED00A27A4E7C04626
:10958000FFFFFF7F37B51300064A05001068046A25
:10959000002C00D1044C0A0000942900FFF770FF52
:1095A0003EBDC04664000020C8000020F8B505009C
:1095B0000E001400002804D08369002B01D100F0B4
:1095C000C1F9224B9C422DD16C68A369A360A38989
:1095D0001B0731D52369002B2ED023682269F7B2EF
:1095E000981A6369F6B2834205DC2100280000F076
:1095F0003BF9002826D1A3680130013BA360236812
:109600005A1C22601F706369834204D0A389DB0760
:109610001AD50A2E18D12100280000F025F90028BB
:1096200012D00FE00A4B9C4201D1AC68CDE7094B48
:109630009C42CAD1EC68C8E72100280000F00CF871
:109640000028CAD0012676423000F8BDF4B50000EB
:1096500014B60000D4B50000364B70B51D68060086
:109660000C00002D05D0AB69002B02D1280000F0C2
:1096700069F9314B9C420FD16C680C23E25E93B2C6
:1096800019072DD4D90611D40923012033603733AB
:109690001343A381404270BD284B9C4201D1AC686A
:1096A000EBE7274B9C42E8D1EC68E6E75B0713D574
:1096B000616B002908D023004433994202D0300066
:1096C000FFF7BEFA002363632422A3899343A38197
:1096D00000236360236923600823A2891343A381C5
:1096E0002369002B0BD1A0218022A389890092003D
:1096F0000B40934203D02100300000F0E1F9012338
:10970000A289134011D00023A36063695B42A36167
:10971000002023698342BED10C23E25E1306BAD532
:1097200040231343A3810138B5E7920700D463694E
:10973000A360EDE764000020F4B5000014B600005B
:10974000D4B5000010B5062000F0E0FB012000F0C9
:109750001DFD0000F7B58A8905000C00130760D4D1
:109760004B68002B04DC0B6C002B01DC0020FEBDE1
:10977000E76A002FFAD000232E682B6080235B015C
:10978000216A1A4034D0606DA3895B0706D56368EF
:10979000C01A636B002B01D0236CC01A0200216A2F
:1097A00000232800E76AB847A189431C06D12B682B
:1097B0001D2B30D82B4ADA40D3072CD50023636009
:1097C00023692360CB0405D5431C02D12B68002BF1
:1097D00000D16065616B2E600029C7D0230044333F
:1097E000994202D02800FFF72BFA00206063BEE701
:1097F00001232800B847431CC6D12B68002BC3D0D7
:109800001D2B01D0162B01D12E60AFE74023A2897A
:109810001343A381ABE740230B430120A3814042C4
:10982000A5E70F69002FA1D00B680F60DB1B019328
:109830000023920700D14B69A360019B002B00DC41
:1098400094E7019B3A00216A2800A66AB0470028E5
:1098500003DC4023A2891343DFE7019B3F181B1A57
:109860000193EAE7010040200B6970B505000C0088
:10987000002B01D1002070BD002804D08369002B8B
:1098800001D100F05FF80B4B9C4209D16C680C22AF
:10989000A35E002BEED021002800FFF75BFFEAE774
:1098A000054B9C4201D1AC68F1E7044B9C42EED1E0
:1098B000EC68ECE7F4B5000014B60000D4B5000085
:1098C000002310B504000360436083608181436618
:1098D000C281036143618361190008225C30FFF794
:1098E000A6F9054B24626362044BA362044BE36256
:1098F000044B236310BDC0464D9F0000759F0000C0
:10990000AD9F0000D99F000010B5024900F08CF80F
:1099100010BDC0466998000070B568254A1E5543C1
:109920000E0029007431FFF7D5F9041E08D000217C
:109930002A00016046600C30A0606832FFF777F9BA
:10994000200070BD836913B50400002B28D1836407
:10995000C3640365134B144A1B68826201939842E7
:1099600001D101238361200000F020F86060200015
:1099700000F01CF8A060200000F018F80022E06061
:1099800004216068FFF79CFF01220921A068FFF70E
:1099900097FF02221221E068FFF792FF0123A361E3
:1099A00013BDC0469CB5000009990000F8B51C4BDA
:1099B00007001E68B369002B02D13000FFF7C2FF19
:1099C0004836B4687368013B04D53368002B07D070
:1099D0003668F6E70C22A55E002D0DD06834F2E75C
:1099E00004213800FFF798FF30600028F0D10C23E5
:1099F00004003B602000F8BD20000A4B656625602E
:109A00006560A560E36025616561A56108222900A4
:109A10005C30FFF70CF96563A563A564E564E9E7CD
:109A20009CB500000100FFFFF7B504000700002609
:109A300001914834002C01D13000FEBD6368A56857
:109A40000093009B013B009301D52468F2E7AB89AA
:109A5000012B08D90E22AB5E013304D02900380057
:109A6000019B984706436835EBE7EC300068704788
:109A700070B50E001D000E23C95E96B014000029BB
:109A800007DA00232B60B3891B0611D48023DB0087
:109A90000FE06A4600F0D8FA0028F2DBF022019BC2
:109AA00012021340054A9B185A4253412B60EDE7BE
:109AB00040230020236016B070BDC04600E0FFFFC9
:109AC000F7B502268B8905000C00334206D023002F
:109AD00047332360236101236361F7BD01AB6A460D
:109AE000FFF7C6FF009907002800FFF7F3F80028EA
:109AF00008D10C22A35E9A05EFD4032293431E43A0
:109B0000A681E4E70F4BAB628023A2892060134358
:109B1000A381009B20616361019B002B0DD00E236C
:109B2000E15E280000F0A2FA002806D00322A389F3
:109B300093431A0001231343A381A0893843A081D2
:109B4000CBE7C0460999000082B0002900D101A9E5
:109B5000101E06D0002B06D013780B601078431E21
:109B6000984102B0704702204042FAE7C9B2821819
:109B7000904201D10020704703788B42FBD0013026
:109B8000F6E710B5884202D98B18984203D3002318
:109B900007E08B5C8354013AFBD210BDCC5CC4540B
:109BA00001339A42FAD1F8E770477047F8B50700D9
:109BB0000D001600002905D11100FFF78BF80400F5
:109BC0002000F8BD002A03D1FFF73AF83400F7E788
:109BD00000F072FA2C00B042F2D231003800FFF7E8
:109BE00079F8041EECD029003200FFF717F829009D
:109BF0003800FFF725F8E3E7F0B58E6885B0070079
:109C00000C00039201939E423CD890238A89DB008A
:109C10001A4234D00325096923685B1A02936369E9
:109C200002985D43EB0F5D19019B6D1001331B180A
:109C3000AB4200D91D00530532D529003800FFF78B
:109C400049F8061E09D10C233B6040230120A2895C
:109C500040421343A38105B0F0BD029A2169FEF78B
:109C6000DDFFA389144A1A4080231343A381029B7A
:109C70002661F61826606561019EED1AA560019BBC
:109C80009E4200D9019E320003992068FFF779FFB8
:109C9000A36800209B1BA36023689E192660DAE757
:109CA0002A003800FFF782FF061EE0D12169380044
:109CB000FEF7C6FFC7E7C0467FFBFFFFF0B59FB0CA
:109CC000029005938B890F0016001B0611D50B69B6
:109CD000002B0ED14021FEF7FDFF386038610028CF
:109CE00005D10C23029A013813601FB0F0BD402348
:109CF0007B61002306AC6361203363761033A37667
:109D000035002B78002B01D0252B46D1AB1B0493BB
:109D10000CD0320039000298FFF76EFF431C00D1CF
:109D2000AEE06269049B9446634463612B78002B28
:109D300000D1A5E0012200235242626002A9543200
:109D400052186E1C2360E360A3601370A365317822
:109D500005225448FFF70AFF751C00281FD122680E
:109D6000D30604D5532302A95B18202119701307C9
:109D700004D5532302A95B182B21197033782A2BA1
:109D800016D0350000210A20E3682A786E1C303A8C
:109D9000092A4ED9002918D010E00135B1E7414B0E
:109DA0002268C01A01238340134323602E00CEE7AC
:109DB000059B191D1B680591002B01DB099304E02D
:109DC0005B42E3600223134323602B782E2B0AD1DE
:109DD0006B782A2B35D1059B02351A1D1B6805921D
:109DE000002B2BDB0793304E297803223000FFF73E
:109DF000BDFE002806D04023801B83402268013529
:109E0000134323602978062228486E1C2176FFF729
:109E1000ADFE00283CD0264B002B25D10722059B08
:109E200007339343083305936369039A9B1863616F
:109E300066E7434301219B183500A6E701235B42F7
:109E4000D0E700230A201A000135636029786E1CD0
:109E50003039092903D9002BC5D00792C3E7424303
:109E6000012352183500F1E705AB00933A00114B7E
:109E70002100029800E000BF0390039B0133D3D17F
:109E8000BB890B985B0600D42FE7012040422CE7EA
:109E900005AB00933A00074B21000298FFF724F925
:109EA000EAE7C046A0B50000A6B50000AAB50000CC
:109EB00000000000F99B000070B504000D001F2990
:109EC00004D9162303600120404270BD436C002B6F
:109ED00004D08A009B181A68002A08D1200000F0DC
:109EE00031F82A000100200000F01AF8EDE7002008
:109EF000012AEAD0511C03D1162301302360E4E784
:109F0000002428001C6090472000DEE710B5034BBA
:109F100001001868FFF7D0FF10BDC04664000020A4
:109F2000002370B5064C050008001100236000F006
:109F3000FFF8431C03D12368002B00D02B6070BDB9
:109F4000C425002010B500F0E3F810BD70B50C007A
:109F50000E25495F00F0B8F8002803DB636D1B187D
:109F6000636570BDA389024A1340A381F9E7C04627
:109F7000FFEFFFFFF8B51F008B8905000C001600EE
:109F8000DB0505D50E23C95E0022022300F080F810
:109F9000A389054A28001340A38132000E23E15E05
:109FA0003B0000F02BF8F8BDFFEFFFFF70B50C0091
:109FB0000E25495F00F06CF8A389421C03D1054AC5
:109FC0001340A38170BD802252011343A3816065B9
:109FD000F8E7C046FFEFFFFF10B50E23C95E00F0A3
:109FE00021F810BD0B1E04D0FF2A04D98A23036078
:109FF0008B3B180070470A700123FAE770B5050023
:10A00000080011000022064C22601A0000F0B6F889
:10A01000431C03D12368002B00D02B6070BDC046C9
:10A02000C4250020002370B5064C050008002360FD
:10A0300000F05EF8431C03D12368002B00D02B6096
:10A0400070BDC046C4250020002370B5064C050035
:10A0500008001100236000F053F8431C03D123686B
:10A06000002B00D02B6070BDC4250020002370B5EC
:10A07000064C05000800236000F052F8431C03D191
:10A080002368002B00D02B6070BDC046C425002083
:10A0900070B50500080011000022064C22601A006D
:10A0A00000F04EF8431C03D12368002B00D02B6036
:10A0B00070BDC046C42500200B1F1B68181F002B55
:10A0C00001DA0B58C018704770B505000800110080
:10A0D0000022064C22601A0000F03AF8431C03D11B
:10A0E0002368002B00D02B6070BDC046C425002023
:10A0F00058220120014B40421A607047C4250020BD
:10A1000058220120014B40421A607047C4250020AC
:10A1100058220120014B40421A607047C42500209C
:10A120005822024B00201A607047C046C425002008
:10A1300058220120014B40421A607047C42500207C
:10A1400058220120014B40421A607047C42500206C
:10A1500058220120014B40421A607047C42500205C
:10A16000044A1368002B00D1034B18181060180024
:10A170007047C04614120020C82500205822012034
:10A18000014B40421A607047C4250020FEE7C046DC
:10A19000F8B5C046F8BC08BC9E467047F8B5C04646
:10A1A000F8BC08BC9E4670475405000064050000DA
:10A1B0007E050000FC050000340600006A06000071
:10A1C000A2060000C80600000407000046070000C1
:10A1D0009C070000E00700004C0800009408000005
:10A1E000BA080000F2080000380900005E0900000B
:10A1F0008C090000BE090000F60900007A0A000080
:10A20000460B0000BC0B0000280C0000700C000086
:10A21000900C0000B20C00008C0D0000D20D00006C
:10A220005405000054050000540500004A0E0000CB
:10A23000B20E0000340F00007A0F0000C20F0000C1
:10A2400040100000BE100000061100004C1100007C
:10A2500082110000C81100000E120000561200000A
:10A26000AA1200000813000046130000B0130000FB
:10A27000E61300002E14000076140000BE14000047
:10A28000F814000040150000881500005405000077
:10A290005405000054050000F015000026160000CB
:10A2A0005C16000088160000BE160000F4160000C0
:10A2B000540500005405000054050000540500003A
:10A2C0002A1700006C170000540500005405000018
:10A2D000B217000002180000281800005405000002
:10A2E00054050000540500005618000086180000B0
:10A2F000B6180000E618000010190000461900000A
:10A300007019000098190000C0190000F019000031
:10A31000201A00004A1A0000741A0000A41A000053
:10A32000E81A000054050000540500005405000020
:10A330005405000054050000181B0000441B0000D9
:10A34000701B00009C1B0000C81B0000FE1B0000CF
:10A35000341C00006A1C0000A01C0000CC1C000083
:10A36000F81C00002E1D00005405000054050000DC
:10A370005405000054050000540500005405000079
:10A380005405000054050000540500005405000069
:10A390005405000054050000540500005405000059
:10A3A0005A1D0000861D000066616C7365007472A2
:10A3B0007565006C697374206F662025642069746C
:10A3C000656D73006F626A656374206F6620636CED
:10A3D0006173733A20256400537461636B20756E5A
:10A3E000646572666C6F7700070000000300000070
:10A3F00032A40000611E00003AA40000651E0000A7
:10A4000043A400005D1E00004CA40000691E000073
:10A410000000000001000000020000000300000036
:10A42000040000000A0000006D6963726F3A6269FF
:10A430007400686173546F6E6500706C6179546F5D
:10A440006E6500686173536572766F00736574534F
:10A450006572766F00496E73756666696369656ECD
:10A4600074206D656D6F727920666F72204D69631F
:10A47000726F426C6F636B73206F626A65637420E6
:10A480006865617000496E73756666696369656EBB
:10A4900074206D656D6F727920666F72204D6963EF
:10A4A000726F426C6F636B7320737461636B000D2A
:10A4B0000A564D2050616E69633A2025730D0A00DB
:10A4C0006D69736300000000D8A40000DD22000065
:10A4D000E1A4000095220000686578546F496E740D
:10A4E0000073696E0000000034A5000049230000DD
:10A4F0003CA500004D23000046A500006B23000092
:10A500004FA50000752300005AA500007F2300001E
:10A5100066A500008923000077A5000093230000B2
:10A520008DA5000057230000A6A5000061230000B0
:10A530006E6574006861735769466900737461726F
:10A5400074576946690073746F705769466900777C
:10A55000696669537461747573006D79495041641B
:10A560006472657373007468696E674465736372BF
:10A57000697074696F6E00636C6561725468696EAE
:10A58000674465736372697074696F6E006170709F
:10A59000656E64546F5468696E674465736372696D
:10A5A0007074696F6E00617070656E64546F54688A
:10A5B000696E6750726F7065727479001A1B1C03A4
:10A5C000040607090A17181903040607090A1718C9
:10A5D00019000000000008080800080A4A400000AE
:10A5E0000A5FEA5FEA0ED92ED36E19324489330C22
:10A5F000924C924D080800000004880808040804E2
:10A60000848488000A448A4000048EC480000000CC
:10A61000048800000EC000000000080001224488E9
:10A62000100C9252524C048C84848E1C824C901ECE
:10A630001EC244924C06CA525FE21FF01EC13E0287
:10A64000448ED12E1FE24488100ED12ED12E0ED171
:10A650002EC4880008000800000480048802448892
:10A660000482000EC00EC008048244880ED126C0A9
:10A67000040ED135B36C0C925ED2521C925C925C8B
:10A680000ED010100E1C9252525C1ED01C901E1E3A
:10A69000D01C90100ED013712E12525ED2521C8814
:10A6A00008081C1FE242524C1254981492101010C9
:10A6B000101E113B75B131113935B3710C925252E4
:10A6C0004C1C925C90100C92524C861C925C9251E5
:10A6D0000ED00C825C1FE4848484125252524C11BE
:10A6E00031312A44113135BB7112524C9252112A28
:10A6F0004484841EC488101E0EC808080E10080466
:10A7000082410EC242424E048A4000000000000016
:10A710001F0804800000000ED2524F10101C925CE3
:10A72000000ED0100E02424ED24E0C925C900E06DD
:10A73000C81C88080ED24EC24C10101C9252080041
:10A74000080808024002424C1014981492080808A5
:10A750000806001B75B131001C925252000C925237
:10A760004C001C925C90000ED24EC2000ED0101015
:10A770000006C8049808080EC807001252524F007D
:10A7800011312A4400113135BB00124C8C9200115A
:10A790002A4498001EC4881E06C48C8486080808B3
:10A7A000080818080C881800000C836000000000DE
:10A7B000010000000200000003000000040000008F
:10A7C000050000000600000007000000080000006F
:10A7D000090000000A0000000B0000000C0000004F
:10A7E0000D0000000E0000000F000000100000002F
:10A7F0001200000014000000160000001800000005
:10A800001A0000001C0000001E00000020000000D4
:10A810002300000026000000290000002C0000009A
:10A820002F00000032000000360000003A00000057
:10A830003E00000042000000460000004B00000007
:10A8400050000000550000005A00000061000000A8
:10A85000680000006F000000760000007D0000002E
:10A86000840000008B0000009200000099000000AE
:10A87000A0000000A7000000AE000000B50000002E
:10A88000BC000000C3000000CA000000D1000000AE
:10A89000D8000000DF000000E6000000ED0000002E
:10A8A000F4000000FB000000FF000000FCA8000016
:10A8B000B923000007A900008528000011A90000A5
:10A8C000992500001EA90000B925000025A9000057
:10A8D000092600002EA90000592600003AA9000010
:10A8E000B12800004BA90000C927000058A90000AA
:10A8F00099270000646973706C6179006C696768FE
:10A90000744C6576656C006D62446973706C617936
:10A91000006D62446973706C61794F6666006D62A8
:10A92000506C6F74006D62556E706C6F74006D6268
:10A93000447261775368617065006D62536861703D
:10A9400065466F724C6574746572006E656F506910
:10A9500078656C53656E64006E656F506978656CE0
:10A9600053657450696E004E6F7420656E6F756725
:10A970006820726F6F6D206576656E206166746504
:10A980007220636F6D70616374696F6E00436F6DE9
:10A9900070616374656420466C61736820636F64E2
:10A9A000652073746F72650A25642062797465731B
:10A9B000207573656420282564252529206F66206D
:10A9C000256400426164207265636F726420666F63
:10A9D000756E6420647572696E6720696E6974694A
:10A9E000616C697A6174696F6E002564202564204A
:10A9F00025642028256420776F72647329002564FC
:10AA0000207265636F7264732C20256420776F72E7
:10AA100064732C206D617849442025642C20636F79
:10AA20006D70616374696F6E206379636C65732008
:10AA30002564005363726970747320636C6561727E
:10AA40006564005374617274656400526573746F59
:10AA50007265642025642073637269707473007278
:10AA60006164696F00000000F6AA0000D5320000A2
:10AA700003AB00004135000013AB0000E5340000DB
:10AA800021AB0000C13600002CAB0000ED3200000D
:10AA90003CAB00006133000050AB0000FD32000011
:10AAA0005FAB0000A13800006BAB00002138000054
:10AAB00074AB0000C53700007FAB00000D3700000D
:10AAC0008AAB00004937000093AB00007D370000DF
:10AAD0009CAB0000113300006E756D626572006EF4
:10AAE0006F6E65006F7468657200706169720073E3
:10AAF0007472696E670064697361626C6552616447
:10AB0000696F006D6573736167655265636569762A
:10AB10006564007061636B65745265636569766531
:10AB2000007061636B657453656E64007265636584
:10AB300069766564496E7465676572007265636500
:10AB4000697665644D6573736167655479706500F6
:10AB50007265636569766564537472696E670073C4
:10AB6000656E64496E74656765720073656E6450E6
:10AB70006169720073656E64537472696E67007305
:10AB800065744368616E6E656C0073657447726FBF
:10AB9000757000736574506F776572007369676EC6
:10ABA000616C537472656E67746800000000000089
:10ABB000963007772C610EEEBA51099919C46D07CA
:10ABC0008FF46A7035A563E9A395649E3288DB0E25
:10ABD000A4B8DC791EE9D5E088D9D2972B4CB60908
:10ABE000BD7CB17E072DB8E7911DBF906410B71DE5
:10ABF000F220B06A4871B9F3DE41BE847DD4DA1A1E
:10AC0000EBE4DD6D51B5D4F4C785D38356986C134E
:10AC1000C0A86B647AF962FDECC9658A4F5C0114C7
:10AC2000D96C0663633D0FFAF50D088DC8206E3BA5
:10AC30005E10694CE44160D5727167A2D1E4033CB7
:10AC400047D4044BFD850DD26BB50AA5FAA8B535DE
:10AC50006C98B242D6C9BBDB40F9BCACE36CD832CD
:10AC6000755CDF45CF0DD6DC593DD1ABAC30D92674
:10AC70003A00DE518051D7C81661D0BFB5F4B42177
:10AC800023C4B3569995BACF0FA5BDB89EB8022874
:10AC90000888055FB2D90CC624E90BB1877C6F2FF9
:10ACA000114C6858AB1D61C13D2D66B69041DC76F4
:10ACB0000671DB01BC20D2982A10D5EF8985B171CD
:10ACC0001FB5B606A5E4BF9F33D4B8E8A2C907787C
:10ACD00034F9000F8EA8099618980EE1BB0D6A7F13
:10ACE0002D3D6D08976C6491015C63E6F4516B6BCC
:10ACF00062616C1CD83065854E0062F2ED95066C81
:10AD00007BA5011BC1F4088257C40FF5C6D9B065F5
:10AD100050E9B712EAB8BE8B7C88B9FCDF1DDD6252
:10AD2000492DDA15F37CD38C654CD4FB5861B24DB8
:10AD3000CE51B53A7400BCA3E230BBD441A5DF4A82
:10AD4000D795D83D6DC4D1A4FBF4D6D36AE9694345
:10AD5000FCD96E34468867ADD0B860DA732D0444F0
:10AD6000E51D03335F4C0AAAC97C0DDD3C7105501B
:10AD7000AA41022710100BBE86200CC925B56857C2
:10AD8000B3856F2009D466B99FE461CE0EF9DE5E0B
:10AD900098C9D9292298D0B0B4A8D7C7173DB359BC
:10ADA000810DB42E3B5CBDB7AD6CBAC02083B8ED4D
:10ADB000B6B3BF9A0CE2B6039AD2B1743947D5EA5A
:10ADC000AF77D29D1526DB048316DC73120B63E389
:10ADD000843B64943E6A6D0DA85A6A7A0BCF0EE4E8
:10ADE0009DFF099327AE000AB19E077D44930FF0A3
:10ADF000D2A3088768F2011EFEC206695D5762F79A
:10AE0000CB67658071366C19E7066B6E761BD4FED6
:10AE1000E02BD3895A7ADA10CC4ADD676FDFB9F9B3
:10AE2000F9EFBE8E43BEB717D58EB060E8A3D6D675
:10AE30007E93D1A1C4C2D83852F2DF4FF167BBD1A3
:10AE40006757BCA6DD06B53F4B36B248DA2B0DD8A6
:10AE50004C1B0AAFF64A0336607A0441C3EF60DF49
:10AE600055DF67A8EF8E6E3179BE69468CB361CB32
:10AE70001A8366BCA0D26F2536E2685295770CCC57
:10AE800003470BBBB91602222F260555BE3BBAC598
:10AE9000280BBDB2925AB42B046AB35CA7FFD7C289
:10AEA00031CFD0B58B9ED92C1DAEDE5BB0C2649B7A
:10AEB00026F263EC9CA36A750A936D02A906099CAD
:10AEC0003F360EEB8567077213570005824ABF9520
:10AED000147AB8E2AE2BB17B381BB60C9B8ED292A3
:10AEE0000DBED5E5B7EFDC7C21DFDB0BD4D2D386FA
:10AEF00042E2D4F1F8B3DD686E83DA1FCD16BE816D
:10AF00005B26B9F6E177B06F7747B718E65A08883D
:10AF1000706A0FFFCA3B06665C0B0111FF9E658FCE
:10AF200069AE62F8D3FF6B6145CF6C1678E20AA078
:10AF3000EED20DD75483044EC2B30339612667A7FE
:10AF4000F71660D04D476949DB776E3E4A6AD1AE4D
:10AF5000DC5AD6D9660BDF40F03BD83753AEBCA9DC
:10AF6000C59EBBDE7FCFB247E9FFB5301CF2BDBD49
:10AF70008AC2BACA3093B353A6A3B4240536D0BA52
:10AF80009306D7CD2957DE54BF67D9232E7A66B3EF
:10AF9000B84A61C4021B685D942B6F2A37BE0BB49C
:10AFA000A18E0CC31BDF055A8DEF022D416C6C2066
:10AFB0007461736B732073746F70706564007630A6
:10AFC000363600202573202573004D656D6F72792C
:10AFD00020636C6561726564004E6F206672656502
:10AFE000207461736B20656E747269657300000074
:10AFF00030B000000D4700003CB00000754A000072
:10B0000042B00000854A000048B00000954A0000A8
:10B010004EB000004147000058B00000A54A0000B3
:10B0200060B000008148000073656E736F7273003A
:10B0300074656D70657261747572650074696C74A5
:10B04000580074696C74590074696C745A00746F98
:10B0500075636852656164006932635265616400BA
:10B06000693263577269746500000000E0B0000047
:10B07000294B0000EEB000002D4B0000F7B000009F
:10B08000394B000001B100003D4B00000AB1000047
:10B09000414B00000FB10000454B000014B100000F
:10B0A000494B000020B100004D4B000027B10000CB
:10B0B000514B000030B10000554B000035B100008D
:10B0C000594B000040B100005D4B00004AB1000048
:10B0D000314B000054B10000354B00007466740021
:10B0E000656E61626C65446973706C617900676557
:10B0F0007457696474680067657448656967687443
:10B1000000736574506978656C006C696E650072D7
:10B1100065637400726F756E646564526563740074
:10B12000636972636C6500747269616E676C650057
:10B130007465787400746674546F75636865640030
:10B14000746674546F7563685800746674546F75D0
:10B1500063685900746674546F75636850726573E0
:10B16000737572650057656C636F6D6520746F2031
:10B170004D6963726F426C6F636B732100705F7314
:10B18000706920213D204E554C4C002F686F6D6535
:10B190002F62726F6D61676F73612F2E706C6174B7
:10B1A000666F726D696F2F7061636B616765732F76
:10B1B0006672616D65776F726B2D61726475696E11
:10B1C0006F6E6F726469636E7266352F6C6962723E
:10B1D00061726965732F5350492F5350492E637024
:10B1E0007000535049436C6173733A3A535049436A
:10B1F0006C617373284E52465F5350495F547970A7
:10B20000652A2C2075696E74385F742C2075696E00
:10B2100074385F742C2075696E74385F742900006F
:10B220000000000000000000654D0000214D0000FE
:10B23000474D0000514D00005B4D0000454D0000A2
:10B2400003000000020000000100000004000000F4
:10B2500005000000110000000C0000000B000000C1
:10B26000120000000A000000060000001A000000A2
:10B270001400000017000000160000001500000078
:10B2800010000000FFFFFFFFFFFFFFFF00000000B6
:10B290001E00000019000000180000000700000058
:10B2A00008000000090000000D0000000E00000072
:10B2B0000F0000001C0000001B0000001D0000002B
:10B2C0001300000000000000000000001552000004
:10B2D0003959000095520000A95200009F52000009
:10B2E0001152000005520000B5520000315200001A
:10B2F0000152000000000000000000000000304388
:10B3000000000000000030C3FB21F93FFB21094091
:10B310007CD91240FB2119407A6A1F407CD9224017
:10B32000BBFD2540FB2129403A462C407A6A2F403C
:10B330005C4731407CD932409C6B3440BBFD35408A
:10B34000DB8F3740FB2139401BB43A403A463C4042
:10B350005AD83D407A6A3F404C7E40405C4741406D
:10B360006C1042407CD942408CA243409C6B4440CC
:10B37000AC344540BBFD4540CBC64640DB8F474023
:10B38000EB584840FB21494083F9A200444E6E002F
:10B39000FC291500D1572700DD34F50062DBC00021
:10B3A0003C999500419043006351FE00BBDEAB0029
:10B3B000B761C5003A6E2400D24D42004906E00054
:10B3C00009EA2E001C92D100EB1DFE0029B11C00E1
:10B3D000E83EA700F535820044BB2E009CE98400BE
:10B3E000B4267000417E5F00D69139005383390046
:10B3F0009CF439008B5F840028F9BD00F81F3B00E6
:10B40000DEFF97000F980500112FEF000A5A8B00FE
:10B410006D1F6D00CF7E360009CB2700464FB70069
:10B420009E663F002DEA5F00BA277500E5EBC70076
:10B430003D7BF100F739070092528A00FB6BEA006E
:10B440001FB15F00085D8D00300356007BFC460095
:10B45000F0AB6B0020BCCF0036F49A00E3A91D00CE
:10B460005E619100081BE60085996500A0145F00ED
:10B470008D40680080D8FF0027734D00060631001C
:10B48000CA561500C9A873007BE260006B8CC0002F
:10B4900000000040FB21F93F000000002D44743EF5
:10B4A000000000809846F83C0000006051CC783BDA
:10B4B00000000080831BF0390000004020257A380E
:10B4C000000000802282E336000000001DF3693591
:10B4D000020000000300000004000000060000005D
:10B4E000A8730000527300005273000080740000C3
:10B4F0004E7300004E7300007674000080740000EC
:10B500004E730000767400004E73000080740000DB
:10B510008474000084740000847400008C74000043
:10B52000A87F0000AA7E0000AA7E0000C88100005B
:10B53000A47E0000A47E0000B0810000C88100004D
:10B54000A47E0000B0810000A47E0000C88100003D
:10B55000BE810000BE810000BE810000CC810000E1
:10B560002C2066756E6374696F6E3A200061737388
:10B57000657274696F6E2022257322206661696C82
:10B5800065643A2066696C6520222573222C206C44
:10B59000696E65202564257325730A006800002004
:10B5A000232D302B2000686C4C00656667454647AC
:10B5B000003031323334353637383941424344452F
:10B5C000460030313233343536373839616263649E
:10B5D00065660000000000000000000000000000A0
:10B5E000000000000000000000000000000000005B
:10B5F000000000000000000000000000000000004B
:10B60000000000000000000000000000000000003A
:10B61000000000000000000000000000000000002A
:10B62000000000000000000000000000000000001A
:10B63000000000004300504F534958002E000020E6
:10B6400020202020202020202828282828202020D2
:10B650002020202020202020202020202020208882
:10B6600010101010101010101010101010101004E6
:10B670000404040404040404041010101010101036
:10B68000414141414141010101010101010101012A
:10B690000101010101010101010110101010101040
:10B6A00042424242424202020202020202020202FA
:10B6B0000202020202020202020210101010200016
:10B6C000000000000000000000000000000000007A
:10B6D000000000000000000000000000000000006A
:10B6E000000000000000000000000000000000005A
:10B6F000000000000000000000000000000000004A
:10B700000000000000000000000000000000000039
:10B710000000000000000000000000000000000029
:10B720000000000000000000000000000000000019
:10B730000000000000000000000000000000000009
:04B740000000000005
:08B74400C449FF7F0100000071
:10B74C00FFFFFFFF400600001800000019FCFFFF80
:10B75C00FFFFFFFFFF0000000200000003000000DD
:10B76C00FFFFFFFF000000000100000000000200CE
:10B77C0001000000FFFFFFFF0000000002000000BE
:10B78C000000040002000000FFFFFFFF00000000AB
:10B79C000300000000000800030000000A00000085
:10B7AC00080000006800002000000000F4B5000054
:10B7BC0014B60000D4B5000000000000000000002A
:10B7CC00000000000000000000000000000000006D
:10B7DC00000000000000000000000000000000005D
:10B7EC00000000000000000000000000000000004D
:10B7FC00000000000000000000000000000000003D
:10B80C0000000000000000004300000000000000E9
:10B81C00000000000000000000000000000000001C
:10B82C0000000000000000004300000000000000C9
:10B83C0000000000000000000000000000000000FC
:10B84C0000000000000000004300000000000000A9
:10B85C0000000000000000000000000000000000DC
:10B86C000000000000000000430000000000000089
:10B87C0000000000000000000000000000000000BC
:10B88C000000000000000000430000000000000069
:10B89C00000000000000000000000000000000009C
:10B8AC000000000000000000430000000000000049
:10B8BC00000000000000000000000000000000007C
:10B8CC000000000000000000430000000000000029
:10B8DC00000000000000000000000000000000005C
:10B8EC000000000000000000E59F0000499B0000E4
:10B8FC00000000003EB600003CB60000BFA40000F3
:10B90C00BFA40000BFA40000BFA40000BFA400009F
:10B91C00BFA40000BFA40000BFA40000BFA400008F
:10B92C00FFFFFFFFFFFFFFFFFFFFFFFFFFFF000019
:10B93C000100415343494900000000000000000091
:10B94C0000000000000000000000000000000000EB
:10B95C000000415343494900000000000000000072
:10B96C0000000000000000000000000000000000CB
:10B97C0000000000E9000000F14C0000395000000C
:08B98C0061550000C10000003C
:04000003000050D5D4
:00000001FF
